:020000040000FA
:040800004DEF0BF0BD
:1008100003B276EF05F0F2B494EF05F09EB09CEFD2
:1008200005F09EB2A4EF05F0F2A81AEF04F0F2B2C0
:1008300025EF04F0F2A620EF04F0F2B022EF04F06E
:10084000FCEF0AF0F296F290FF00CD90F2929EA09B
:100850002FEF04F00101533F2FEF04F0542BAEC1F2
:10086000B2F1AFC1B3F1B0C1B4F1B1C1B5F1AAC138
:10087000AEF1ABC1AFF1ACC1B0F1ADC1B1F1A6C148
:10088000AAF1A7C1ABF1A8C1ACF1A9C1ADF1A2C158
:10089000A6F1A3C1A7F1A4C1A8F1A5C1A9F19EC168
:1008A000A2F19FC1A3F1A0C1A4F1A1C1A5F19AC178
:1008B0009EF19BC19FF19CC1A0F19DC1A1F196C188
:1008C0009AF197C19BF198C19CF199C19DF1CECF4E
:1008D00096F1CFCF97F153C198F154C199F1CF6AF6
:1008E000CE6A0101536B546B9E90CD800FBC0F8E6E
:1008F0000FBA7EEF04F00F8AFCEF0AF00F8C0FBEE8
:10090000BAEF04F096C19AF197C19BF198C19CF19E
:1009100099C19DF19AC19EF19BC19FF19CC1A0F12B
:100920009DC1A1F19EC1A2F19FC1A3F1A0C1A4F1FB
:10093000A1C1A5F1A2C1A6F1A3C1A7F1A4C1A8F1CB
:10094000A5C1A9F1A6C1AAF1A7C1ABF1A8C1ACF19B
:10095000A9C1ADF1AAC1AEF1ABC1AFF1ACC1B0F16B
:10096000ADC1B1F1AEC1B2F1AFC1B3F1B0C1B4F13B
:10097000B1C1B5F101015E6B5F6B606B616B96514C
:100980005E2797515F2398516023995161239A51B3
:100990005E279B515F239C5160239D5161239E5193
:1009A0005E279F515F23A0516023A1516123A25173
:1009B0005E27A3515F23A4516023A5516123A65153
:1009C0005E27A7515F23A8516023A9516123AA5133
:1009D0005E27AB515F23AC516023AD516123AE5113
:1009E0005E27AF515F23B0516023B1516123B251F3
:1009F0005E27B3515F23B4516023B5516123D89072
:100A00000101613360335F335E33D890010161339C
:100A100060335F335E33D8900101613360335F33FD
:100A20005E3300C10CF101C10DF102C10EF103C131
:100A30000FF104C110F105C111F106C112F107C196
:100A400013F108C114F109C115F10AC116F10BC166
:100A500017F134C135F111B839EF05F00101620E1B
:100A6000046F010E056F000E066F000E076F42EF58
:100A700005F00101A70E046F020E056F000E066F50
:100A8000000E076F5EC100F15FC101F160C102F1AC
:100A900061C103F1D4EC2BF003BF04D018BE02D027
:100AA00018A0108C11A05AEF05F010BA5AEF05F0FB
:100AB0000F80108A0CC100F10DC101F10EC102F1CD
:100AC0000FC103F110C104F111C105F112C106F10A
:100AD00013C107F114C108F115C109F116C10AF1DA
:100AE00017C10BF135C134F1FCEF0AF00392ABB240
:100AF000AB98AB88030103EE00F080517F0BE92631
:100B000004C0EFFF802B8151805D700BD8A48B82D5
:100B100000008051815D700BD8A48B9281518019A7
:100B2000D8B40790FCEF0AF0F2940101453FFCEFC6
:100B30000AF0462BFCEF0AF09E900101533FFCEFB8
:100B40000AF0542BFCEF0AF09E9211B821EF08F046
:100B5000040066A1ACEF05F08BB4B6EF05F010AC65
:100B6000B6EF05F08B84109CB7EF05F08B94077CF3
:100B700007ACD2EF05F0C274C2B4CCEF05F0C3CF1E
:100B8000B7F5C4CFB8F50501D890B833B733D890CE
:100B9000B833B733D3EF05F0C3CF55F1C4CF56F117
:100BA000D3EF05F0C28207B440EF06F047C14BF126
:100BB00048C14CF149C14DF14AC14EF15EC162F1EB
:100BC0005FC163F160C164F161C165F196C1B6F1C5
:100BD00097C1B7F198C1B8F199C1B9F19AC1BAF109
:100BE0009BC1BBF19CC1BCF19DC1BDF19EC1BEF1D9
:100BF0009FC1BFF1A0C1C0F1A1C1C1F1A2C1C2F1A9
:100C0000A3C1C3F1A4C1C4F1A5C1C5F1A6C1C6F178
:100C1000A7C1C7F1A8C1C8F1A9C1C9F1AAC1CAF148
:100C2000ABC1CBF1ACC1CCF1ADC1CDF1AEC1CEF118
:100C3000AFC1CFF1B0C1D0F1B1C1D1F1B2C1D2F1E8
:100C4000B3C1D3F1B4C1D4F1B5C1D5F1B7C5B9F5CC
:100C5000B8C5BAF5B9C5BBF5BAC5BCF50101555162
:100C60005B2756515C23E86A5D230E2E40EF06F0A9
:100C70005CC157F15DC158F15B6B5C6B5D6B078EBE
:100C80000201002FFCEF0AF03C0E006F1950E00B40
:100C9000E00AE866128817BE02D017B4108E00C1B1
:100CA0000CF101C10DF102C10EF103C10FF104C13C
:100CB00010F105C111F106C112F107C113F108C10C
:100CC00014F109C115F10AC116F10BC117F134C1B4
:100CD00035F105012F51000AD8B41AEF07F00501CC
:100CE0002F51010AD8B4A4EF06F005012F51020AD2
:100CF000D8B4E5EF06F005012F51030AD8B4E5EFAB
:100D000006F005012F51040AD8B4E5EF06F00501FD
:100D10002F51050AD8B4E5EF06F005012F51060A58
:100D2000D8B4E5EF06F005012F51070AD8B4E5EF76
:100D300006F005012F51320AD8B4A2EF06F02F6B4E
:100D40001AEF07F01AEF07F005015767AFEF06F04B
:100D50005867AFEF06F05967AFEF06F05A67B3EF89
:100D600006F01AEF07F05BC500F15CC501F15DC547
:100D700002F15EC503F10101010E046F000E056F63
:100D8000000E066F000E076FD4EC2BF000C15BF570
:100D900001C15CF502C15DF503C15EF50067D8EFE6
:100DA00006F00167D8EF06F00267D8EF06F0036798
:100DB0001AEF07F057C55BF558C55CF559C55DF5E9
:100DC0005AC55EF50F881AEF07F005013067EBEFA3
:100DD00006F01AEF07F00FBE00EF07F010A005EFC6
:100DE00007F001014767FCEF06F04867FCEF06F0EB
:100DF0004967FCEF06F04A6700EF07F005EF07F0E0
:100E000007AE05EF07F017EF07F00501312F1AEFD6
:100E100007F03C0E316F302F1AEF07F00101000E82
:100E2000626FE00E636FA50E646F010E656F0501C2
:100E3000306B0F880501666B37B720EF07F06681CE
:100E40000CC100F10DC101F10EC102F10FC103F19E
:100E500010C104F111C105F112C106F113C107F16E
:100E600014C108F115C109F116C10AF117C10BF13E
:100E700035C134F100C10CF101C10DF102C10EF117
:100E800003C10FF104C110F105C111F106C112F146
:100E900007C113F108C114F109C115F10AC116F116
:100EA0000BC117F134C135F101018A675FEF07F01B
:100EB0008B675FEF07F08C675FEF07F08D6763EF7D
:100EC00007F093EF07F08EC100F18FC101F190C1DF
:100ED00002F191C103F10101010E046F000E056FD3
:100EE000000E066F000E076FD4EC2BF000C18EF1E0
:100EF00001C18FF102C190F103C191F1006788EF48
:100F000007F0016788EF07F0026788EF07F00367D3
:100F100093EF07F08AC18EF18BC18FF18CC190F1F4
:100F20008DC191F10F80D57ED5BE6DD0D6CF47F162
:100F3000D7CF48F145C149F1E86AE8CF4AF118BE78
:100F400002D018A0108C109047C100F148C101F1E7
:100F500049C102F14AC103F101010A0E046F000EFA
:100F6000056F000E066F000E076FD4EC2BF003AF79
:100F70001080010154A7C9EF07F00F9A0F9C0F9E34
:100F80000101000E5E6F600E5F6F3D0E606F080E18
:100F9000616F010147BFD9EF07F04867D9EF07F04C
:100FA0004967D9EF07F04A67D9EF07F0F288FEEFFB
:100FB00007F0F2985E6B5F6B606B616B966B976B83
:100FC000986B996B9A6B9B6B9C6B9D6B9E6B9F6BED
:100FD000A06BA16BA26BA36BA46BA56BA66BA76B9D
:100FE000A86BA96BAA6BAB6BAC6BAD6BAE6BAF6B4D
:100FF000B06BB16BB26BB36BB46BB56BD76AD66ABF
:101000000101456B466B0CC100F10DC101F10EC130
:1010100002F10FC103F110C104F111C105F112C1B8
:1010200006F113C107F114C108F115C109F116C188
:101030000AF117C10BF135C134F1FCEF0AF0FCEFF6
:101040000AF00201002F65EF0AF0D59ED6CF47F1D6
:10105000D7CF48F145C149F1E86AE8CF4AF1D76AEC
:10106000D66A0101456B466BD58E1950E00BE00A3C
:10107000E866128817BE02D017B4108E16AE1B8C0D
:1010800000C10CF101C10DF102C10EF103C10FF15C
:1010900004C110F105C111F106C112F107C113F12C
:1010A00008C114F109C115F10AC116F10BC117F1FC
:1010B00034C135F10FA0109A11B86AEF08F00101A0
:1010C000620E046F010E056F000E066F000E076FB3
:1010D00073EF08F00101A70E046F020E056F000EFA
:1010E000066F000E076F47C100F148C101F149C109
:1010F00002F14AC103F1D4EC2BF003BF86EF08F0F4
:1011000018BE02D018A0108C11B00F800CC100F1D5
:101110000DC101F10EC102F10FC103F110C104F1C3
:1011200011C105F112C106F113C107F114C108F193
:1011300015C109F116C10AF117C10BF135C134F11E
:1011400002013C0E006F00C10CF101C10DF102C1A2
:101150000EF103C10FF104C110F105C111F106C177
:1011600012F107C113F108C114F109C115F10AC147
:1011700016F10BC117F134C135F105012F51000AE9
:10118000D8B46EEF09F005012F51010AD8B4F8EF79
:1011900008F005012F51020AD8B439EF09F0050112
:1011A0002F51030AD8B439EF09F005012F51040A71
:1011B000D8B439EF09F005012F51050AD8B439EF39
:1011C00009F005012F51060AD8B439EF09F00501DD
:1011D0002F51070AD8B439EF09F005012F51320A0F
:1011E000D8B4F6EF08F02F6B6EEF09F06EEF09F050
:1011F0000501576703EF09F0586703EF09F05967D6
:1012000003EF09F05A6707EF09F06EEF09F05BC5CD
:1012100000F15CC501F15DC502F15EC503F101019C
:10122000010E046F000E056F000E066F000E076FB3
:10123000D4EC2BF000C15BF501C15CF502C15DF59A
:1012400003C15EF500672CEF09F001672CEF09F090
:1012500002672CEF09F003676EEF09F057C55BF5E5
:1012600058C55CF559C55DF55AC55EF50F886EEF3A
:1012700009F0050130673FEF09F06EEF09F00FBE8E
:1012800054EF09F010A059EF09F00101476750EF42
:1012900009F0486750EF09F0496750EF09F04A67D5
:1012A00054EF09F059EF09F007AE59EF09F06BEF71
:1012B00009F00501312F6EEF09F03C0E316F302F30
:1012C0006EEF09F00101000E626FE00E636FA50E74
:1012D000646F010E656F0501306B0F880501666B49
:1012E00037B774EF09F066810CC100F10DC101F14F
:1012F0000EC102F10FC103F110C104F111C105F1DA
:1013000012C106F113C107F114C108F115C109F1A9
:1013100016C10AF117C10BF135C134F100C10CF14E
:1013200001C10DF102C10EF103C10FF104C110F1B1
:1013300005C111F106C112F107C113F108C114F181
:1013400009C115F10AC116F10BC117F134C135F10C
:1013500001018A67B3EF09F08B67B3EF09F08C677F
:10136000B3EF09F08D67B7EF09F0E7EF09F08EC131
:1013700000F18FC101F190C102F191C103F10101AE
:10138000010E046F000E056F000E066F000E076F52
:10139000D4EC2BF000C18EF101C18FF102C190F1AC
:1013A00003C191F10067DCEF09F00167DCEF09F0A0
:1013B0000267DCEF09F00367E7EF09F08AC18EF1FD
:1013C0008BC18FF18CC190F18DC191F10F80109084
:1013D00047C100F148C101F149C102F14AC103F11D
:1013E00001010A0E046F000E056F000E066F000E5D
:1013F000076FD4EC2BF003AF1080010154A70DEF61
:101400000AF00F9A0F9C0F9E0101000E5E6F600E96
:101410005F6F3D0E606F080E616F47C100F148C1FC
:1014200001F149C102F14AC103F10101140E046F37
:10143000050E056F000E066F000E076FD4EC2BF043
:1014400003AF26EF0AF0F2884BEF0AF0F2985E6BDA
:101450005F6B606B616B966B976B986B996B9A6B1C
:101460009B6B9C6B9D6B9E6B9F6BA06BA16BA26B30
:10147000A36BA46BA56BA66BA76BA86BA96BAA6BE0
:10148000AB6BAC6BAD6BAE6BAF6BB06BB16BB26B90
:10149000B36BB46BB56B0CC100F10DC101F10EC1A2
:1014A00002F10FC103F110C104F111C105F112C124
:1014B00006F113C107F114C108F115C109F116C1F4
:1014C0000AF117C10BF135C134F104008BB470EF90
:1014D0000AF010AC70EF0AF08B84109C71EF0AF0E8
:1014E0008B94077C07AC8CEF0AF0C274C2B486EF11
:1014F0000AF0C3CFB7F5C4CFB8F50501D890B8331B
:10150000B733D890B833B7338DEF0AF0C3CF55F166
:10151000C4CF56F18DEF0AF0C28207B4FAEF0AF099
:1015200047C14BF148C14CF149C14DF14AC14EF19F
:101530005EC162F15FC163F160C164F161C165F1D7
:1015400096C1B6F197C1B7F198C1B8F199C1B9F197
:101550009AC1BAF19BC1BBF19CC1BCF19DC1BDF167
:101560009EC1BEF19FC1BFF1A0C1C0F1A1C1C1F137
:10157000A2C1C2F1A3C1C3F1A4C1C4F1A5C1C5F107
:10158000A6C1C6F1A7C1C7F1A8C1C8F1A9C1C9F1D7
:10159000AAC1CAF1ABC1CBF1ACC1CCF1ADC1CDF1A7
:1015A000AEC1CEF1AFC1CFF1B0C1D0F1B1C1D1F177
:1015B000B2C1D2F1B3C1D3F1B4C1D4F1B5C1D5F147
:1015C000B7C5B9F5B8C5BAF5B9C5BBF5BAC5BCF567
:1015D000010155515B2756515C23E86A5D230E2EAD
:1015E000FAEF0AF05CC157F15DC158F15B6B5C6BBF
:1015F0005D6B078EFCEF0AF002C0E0FF005001C0F7
:10160000D8FF1000A6B202EF0BF00CC0A9FF0BC070
:10161000A8FFA69EA69CA684F29E550EA76EAA0EB3
:10162000A76EA682F28EA694A6B214EF0BF00C2A37
:101630001200A96EA69EA69CA680A8500C2A120095
:1016400004012C0E826F6DEC0EF0CFEC2CF00C50E0
:1016500019EC0BF0E8CF00F10C5019EC0BF0E8CFCF
:1016600001F101AF39EF0BF00101FF0E026FFF0E28
:10167000036F72EC2CF0296745EF0BF00401200E8C
:10168000826F6DEC0EF04AEF0BF004012D0E826FAD
:101690006DEC0EF09CEC2AF01200076A0F6A106ADB
:1016A000116A126A0F010D0EC16E860EC06E030E16
:1016B000C26E0F01680E896E130E926E080E8A6E4E
:1016C000F30E936E8B6A900E946EC80E19EC0BF0AD
:1016D000E8CFE8FF1098E8A0108810A805D00E0EFB
:1016E000216E8E0E226E04D00F0E216E8F0E226E92
:1016F0004EEC2DF0F18EF19EFC0E19EC0BF0E8CFC4
:101700000BF00BA011800BA211820BA411840BA86B
:101710001188C90E19EC0BF0E8CF16F0CA0E19ECBF
:101720000BF0E8CF17F0CB0E19EC0BF0E8CF18F068
:10173000CC0E19EC0BF0E8CF19F0CD0E19EC0BF034
:10174000E8CF2EF01B6A1C6A0E6A01015B6B5C6BB2
:101750005D6B576B586BF29A0101476B486B496B95
:101760004A6B4B6B4C6B4D6B4E6B4F6B506B516BB5
:10177000526B456B466BD76AD66A0F01280ED56E41
:10178000F28A9D90B00ECD6E01015E6B5F6B606B57
:10179000616B626B636B646B656B666B676B686BCD
:1017A000696B536B546BCF6ACE6A0F9A0F9C0F9E76
:1017B0009D80760ECA6E9D8202013C0E006FCC6A3F
:1017C000160E19EC0BF0E8CF00F1170E19EC0BF028
:1017D000E8CF01F1180E19EC0BF0E8CF02F1190E69
:1017E00019EC0BF0E8CF03F1010103AF12EF0CF09D
:1017F000CFEC2CF0160E0C6E00C10BF002EC0BF0CF
:10180000170E0C6E01C10BF002EC0BF0180E0C6EF3
:1018100002C10BF002EC0BF0190E0C6E03C10BF0C1
:1018200002EC0BF000C18AF101C18BF102C18CF115
:1018300003C18DF100C18EF101C18FF102C190F1A0
:1018400003C191F11A0E19EC0BF0E8CF00F11B0E59
:1018500019EC0BF0E8CF01F11C0E19EC0BF0E8CFFE
:1018600002F11D0E19EC0BF0E8CF03F1010103AFFB
:1018700068EF0CF0CFEC2CF01A0E0C6E00C10BF0E0
:1018800002EC0BF01B0E0C6E01C10BF002EC0BF026
:101890001C0E0C6E02C10BF002EC0BF01D0E0C6E58
:1018A00003C10BF002EC0BF01A0E19EC0BF0E8CFB1
:1018B00000F11B0E19EC0BF0E8CF01F11C0E19EC36
:1018C0000BF0E8CF02F11D0E19EC0BF0E8CF03F19D
:1018D00000C192F101C193F102C194F103C195F1EC
:1018E000240EAC6E900EAB6E240EAC6E080EB86E6D
:1018F000000EB06E1F0EAF6E0401806B816B0F0186
:10190000900EAB6E0F019D8A0301806B816BC26BE1
:101910008B92D6EC31F0D6EC31F032EC33F0B5EC02
:101920002FF0200E19EC0BF0E8CF2FF505012F5109
:10193000FF0AD8A4A3EF0CF02F6B200E0C6E2FC55E
:101940000BF002EC0BF00501010E306F3C0E316F15
:10195000250E19EC0BF0E8CF00F1260E19EC0BF078
:10196000E8CF01F1270E19EC0BF0E8CF02F1280EB9
:1019700019EC0BF0E8CF03F1010103AFDAEF0CF043
:10198000CFEC2CF0250E0C6E00C10BF002EC0BF02E
:10199000260E0C6E01C10BF002EC0BF0270E0C6E44
:1019A00002C10BF002EC0BF0280E0C6E03C10BF021
:1019B00002EC0BF000C157F501C158F502C159F511
:1019C00003C15AF500C15BF501C15CF502C15DF5CB
:1019D00003C15EF5290E19EC0BF0E8CF5FF50501A8
:1019E00060515F5DD8A05FC560F505012F51020A07
:1019F0000EE181B807EF0DF00501602F04EF0DF047
:101A00005FC560F507EF0DF081BA71EF33F0210E7D
:101A100019EC0BF0E8CF00F1220E19EC0BF0E8CF37
:101A200001F1230E19EC0BF0E8CF02F1240E19ECB2
:101A30000BF0E8CF03F1010103AF4DEF0DF0CFEC58
:101A40002CF0210E0C6E00C10BF002EC0BF0220EFC
:101A50000C6E01C10BF002EC0BF0230E0C6E02C1F8
:101A60000BF002EC0BF0240E0C6E03C10BF002EC39
:101A70000BF0210E19EC0BF0E8CF00F1220E19EC5F
:101A80000BF0E8CF01F1230E19EC0BF0E8CF02F1D7
:101A9000240E19EC0BF0E8CF03F100C161F501C190
:101AA00062F502C163F503C164F5FDEC2EF0FFECB5
:101AB0002DF057EC2DF005012F51030A12E005011E
:101AC0002F51040A1DE005012F51050A24E00501EC
:101AD0002F51060A32E005012F51070A38E0B0EF16
:101AE0000DF0B0C500F101010F0E0017010100510A
:101AF000000A36E001010051050A32E0ADEF0DF0B9
:101B0000B0C500F101010F0E001701010051000ADC
:101B100027E0ADEF0DF00501B051000A21E005010D
:101B2000B051150A1DE00501B051300A19E0050158
:101B3000B051450A15E0ADEF0DF00501B051000AB6
:101B40000FE00501B051300A0BE0ADEF0DF00501DB
:101B5000B051000A05E0ADEF0DF081BA71EF33F03E
:101B600007900001F28EF28C12AE03D012BC83EF0C
:101B700018F007B01EEF29F00FB0BAEF22F010BE38
:101B8000BAEF22F012B8BAEF22F00FB857EF1CF0FC
:101B90000301805181197F0BD8B41EEF29F013EE99
:101BA00000F081517F0BE126812BE7CFE8FFE00BAE
:101BB000D8B41EEF29F023EE82F0C2513F0BD92694
:101BC000E7CFDFFFC22BDF50780AD8A41EEF29F041
:101BD00007808EC100F18FC101F190C102F191C166
:101BE00003F10101040E046F000E056F000E066F75
:101BF000000E076FD4EC2BF000AF08EF0EF00101E0
:101C0000030E8E6F000E8F6F000E906F000E916F9F
:101C100003018251720AD8B49FEF22F08251520A16
:101C2000D8B49FEF22F08251750AD8B49FEF22F00A
:101C30008251630AD8B4D8EF25F08251690AD8B42A
:101C40004EEF1FF082517A0AD8B461EF20F0825132
:101C5000490AD8B4EDEF1EF08251500AD8B40BEF08
:101C60001EF08251700AD8B44EEF1EF08251540A11
:101C7000D8B479EF1EF08251740AD8B4BFEF1EF0C9
:101C80008251410AD8B483EF0FF082514B0AD8B485
:101C900081EF0EF082516D0AD8B48DEF13F08251AE
:101CA0004D0AD8B4A6EF13F08251730AD8B4CFEF1F
:101CB00021F08251530AD8B434EF22F082514C0AF9
:101CC000D8B435EF14F08251590AD8B4DEEF12F0CF
:101CD00012AE01D0128C0FEF26F0040114EE00F0CA
:101CE00080517F0BE12682C4E7FF802B12000401A4
:101CF0000D0E826F6DEC0EF00A0E826F6DEC0EF021
:101D0000120004014B0E826F6DEC0EF004012C0EDC
:101D1000826F6DEC0EF081B802D02EB630D0030188
:101D20008351430AD8B4C6EF0EF003018351630A0E
:101D3000D8B4C8EF0EF003018351520AD8B4CAEFE9
:101D40000EF003018351720AD8B4CCEF0EF00301F8
:101D50008351470AD8B4CEEF0EF003018351670ACE
:101D6000D8B4D0EF0EF003018351540AD8B4D2EFA7
:101D70000EF003018351740AD8B441EF0FF0030150
:101D80008351550AD8B4D4EF0EF082D02E807AD089
:101D90002E9078D02E8276D02E9274D02E8472D04F
:101DA0002E9470D02E866ED084C330F185C331F16D
:101DB00086C332F187C333F10101296B1DEC2DF08D
:101DC00094EC2CF000C104F101C105F102C106F14F
:101DD00003C107F110EC2DF0200EF86EF76AF66AD9
:101DE0000900F5CF2CF10900F5CF2DF10900F5CF51
:101DF0002EF10900F5CF2FF10900F5CF30F10900E0
:101E0000F5CF31F10900F5CF32F10900F5CF33F10B
:101E10000101296B1DEC2DF094EC2CF0D4EC2BF08F
:101E200000671AEF0FF001671AEF0FF002671AEF61
:101E30000FF0036701D025D004014E0E826F6DECC8
:101E40000EF004016F0E826F6DEC0EF004014D0E6A
:101E5000826F6DEC0EF00401610E826F6DEC0EF07E
:101E60000401740E826F6DEC0EF00401630E826F3C
:101E70006DEC0EF00401680E826F6DEC0EF00DEF4C
:101E800026F02E96CD0E0C6E2EC00BF002EC0BF051
:101E9000CD0E19EC0BF0E8CF2EF02EB006D00401D9
:101EA000630E826F6DEC0EF005D00401430E826F5D
:101EB0006DEC0EF02EB206D00401720E826F6DEC46
:101EC0000EF005D00401520E826F6DEC0EF02EB4B0
:101ED00006D00401670E826F6DEC0EF005D0040190
:101EE000470E826F6DEC0EF02EB606D00401740E14
:101EF000826F6DEC0EF005D00401540E826F6DEC14
:101F00000EF00DEF26F00401410E826F6DEC0EF025
:101F100003018351310AD8B4FEEF11F0030183515C
:101F2000320AD8B42EEF11F003018351330AD8B42A
:101F3000B7EF10F003018351340AD8B4A7EF0FF0C4
:101F400004013F0E826F6DEC0EF00DEF26F0CC0E0B
:101F500019EC0BF0E8CF0BF004012C0E826F6DEC46
:101F60000EF003018451310AD8B4CBEF0FF0030116
:101F70008451300AD8B4CDEF0FF0030184514D0ADB
:101F8000D8B4D7EF0FF003018451540AD8B4DEEF70
:101F90000FF0F5EF0FF08A8401D08A940BAE04D0D5
:101FA0000BAC02D00BBA21D0E00E0B1218D01F0ED2
:101FB0000B168539E844E00B0B1211D0E00E0B161E
:101FC00010EC2DF085C332F186C333F10101296B8A
:101FD0001DEC2DF094EC2CF000511F0B0B12CC0ECD
:101FE0000C6E0BC00BF002EC0BF00401340E826F90
:101FF0006DEC0EF004012C0E826F6DEC0EF0CC0E29
:1020000019EC0BF0E8CF19F08AB406D00401300EB9
:10201000826F6DEC0EF005D00401310E826F6DEC15
:102020000EF004012C0E826F6DEC0EF01938E840B2
:10203000070BE8CF82F40401300E82276DEC0EF01E
:1020400004012C0E826F6DEC0EF0CFEC2CF01950C9
:102050001F0BE8CF00F172EC2CF032C182F40401C6
:10206000300E82276DEC0EF033C182F40401300E85
:1020700082276DEC0EF004012C0E826F6DEC0EF0D9
:10208000CFEC2CF02CC000F100AF0BD0FF0E016F95
:10209000FF0E026FFF0E036F04012D0E826F6DECB9
:1020A0000EF072EC2CF031C182F40401300E822764
:1020B0006DEC0EF032C182F40401300E82276DEC1B
:1020C0000EF033C182F40401300E82276DEC0EF065
:1020D00004012C0E826F6DEC0EF0CFEC2CF02BC0B7
:1020E00000F172EC2CF031C182F40401300E822731
:1020F0006DEC0EF032C182F40401300E82276DECDB
:102100000EF033C182F40401300E82276DEC0EF024
:1021100004012C0E826F6DEC0EF0CFEC2CF02DC074
:1021200000F100AF0BD0FF0E016FFF0E026FFF0E2C
:10213000036F04012D0E826F6DEC0EF072EC2CF02B
:1021400031C182F40401300E82276DEC0EF032C1F1
:1021500082F40401300E82276DEC0EF033C182F45C
:102160000401300E82276DEC0EF00DEF26F0CB0E41
:1021700019EC0BF0E8CF0BF004012C0E826F6DEC24
:102180000EF003018451450AD8B4DBEF10F00301CF
:102190008451440AD8B4DEEF10F003018451300AB0
:1021A000D8B4E1EF10F003018451310AD8B4E5EF5F
:1021B00010F0F0EF10F00B9EEAEF10F00B8EEAEF4C
:1021C00010F0FC0E0B16EAEF10F0FC0E0B160B8055
:1021D000EAEF10F0CB0E0C6E0BC00BF002EC0BF024
:1021E0000401330E826F6DEC0EF004012C0E826F31
:1021F0006DEC0EF0CB0E19EC0BF0E8CF18F018BE1A
:1022000009EF11F00401450E826F6DEC0EF00EEF38
:1022100011F00401440E826F6DEC0EF004012C0EDF
:10222000826F6DEC0EF00401300E826F6DEC0EF0DB
:1022300004012C0E826F6DEC0EF018B027EF11F038
:102240000401300E826F6DEC0EF02CEF11F00401E2
:10225000310E826F6DEC0EF00DEF26F0CA0E19EC08
:102260000BF0E8CF0BF004012C0E826F6DEC0EF03A
:1022700003018451450AD8B46AEF11F00301845177
:10228000440AD8B46DEF11F0030184514D0AD8B45B
:1022900076EF11F003018451410AD8B470EF11F0C8
:1022A00003018451460AD8B473EF11F0030184513D
:1022B000560AD8B47EEF11F003018451500AD8B405
:1022C00089EF11F003018451520AD8B48CEF11F058
:1022D00095EF11F00B9E8FEF11F00B8E8FEF11F039
:1022E0000B9C8FEF11F00B8C8FEF11F0FC0E0B1687
:1022F00085C3E8FF030B0B128FEF11F0C70E0B160F
:1023000085C3E8FF070BE846E846E8460B128FEF67
:1023100011F00B848FEF11F00B948FEF11F0CA0EB8
:102320000C6E0BC00BF002EC0BF0CA0E19EC0BF0AC
:10233000E8CF17F00401320E826F6DEC0EF004014D
:102340002C0E826F6DEC0EF017BEAEEF11F0040193
:10235000450E826F6DEC0EF0B3EF11F00401440EE8
:10236000826F6DEC0EF004012C0E826F6DEC0EF09E
:1023700017C0E8FF030BE8CF82F40401300E822778
:102380006DEC0EF004012C0E826F6DEC0EF017BC9C
:10239000D1EF11F00401410E826F6DEC0EF0D6EF1B
:1023A00011F00401460E826F6DEC0EF004012C0E4C
:1023B000826F6DEC0EF017C0E8FF380BE842E84280
:1023C000E842E8CF82F40401300E82276DEC0EF073
:1023D00004012C0E826F6DEC0EF017B4F7EF11F0C4
:1023E0000401520E826F6DEC0EF0FCEF11F004014F
:1023F000500E826F6DEC0EF00DEF26F0C90E19EC49
:102400000BF0E8CF0BF004012C0E826F6DEC0EF098
:1024100003018451450AD8B41CEF12F00301845122
:10242000440AD8B41FEF12F0030184514D0AD8B406
:1024300022EF12F030EF12F00B9E2AEF12F00B8E0B
:102440002AEF12F0F80E0B1685C3E8FF070B0B12EC
:102450002AEF12F0C90E0C6E0BC00BF002EC0BF061
:102460000401310E826F6DEC0EF004012C0E826FB0
:102470006DEC0EF0C90E19EC0BF0E8CF16F016BE9D
:1024800006D00401450E826F6DEC0EF005D00401FC
:10249000440E826F6DEC0EF004012C0E826F6DEC19
:1024A0000EF016C0E8FF070BE8CF82F40401300EEF
:1024B00082276DEC0EF004012C0E826F6DEC0EF095
:1024C0000780CFEC2CF027C0E8FF003B004300431F
:1024D000030B72EC2CF033C182F40401300E82271E
:1024E0006DEC0EF004012C0E826F6DEC0EF0CFEC53
:1024F0002CF027C001F1019F019D28C000F10101CE
:1025000072EC2CF02FC182F40401300E82276DECA6
:102510000EF030C182F40401300E82276DEC0EF013
:1025200031C182F40401300E82276DEC0EF032C10D
:1025300082F40401300E82276DEC0EF033C182F478
:102540000401300E82276DEC0EF004012C0E826F18
:102550006DEC0EF0CFEC2CF029C001F12AC000F197
:10256000D89001330033D89001330033010172EC6D
:102570002CF02FC182F40401300E82276DEC0EF096
:1025800030C182F40401300E82276DEC0EF031C1AF
:1025900082F40401300E82276DEC0EF032C182F419
:1025A0000401300E82276DEC0EF033C182F4040179
:1025B000300E82276DEC0EF00DEF26F0FC0E19ECBC
:1025C0000BF0E8CF0BF003018351520AD8B415EF9A
:1025D00013F003018351720AD8B418EF13F003010A
:1025E0008351500AD8B41BEF13F003018351700AD2
:1025F000D8B41EEF13F003018351550AD8B421EF6C
:1026000013F003018351750AD8B424EF13F00301CA
:102610008351430AD8B42DEF13F003018351630AA9
:10262000D8B430EF13F039EF13F00B9033EF13F011
:102630000B8033EF13F00B9233EF13F00B8233EF79
:1026400013F00B9433EF13F00B8433EF13F00B966E
:1026500033EF13F00B8633EF13F00B9833EF13F0D7
:102660000B8833EF13F0FC0E0C6E0BC00BF002EC7A
:102670000BF00401590E826F6DEC0EF01190119267
:1026800011941198FC0E19EC0BF0E8CF0BF00BA095
:1026900011800BA211820BA411840BA8118811A028
:1026A00059EF13F00401520E826F6DEC0EF05EEFE5
:1026B00013F00401720E826F6DEC0EF011A868EF3A
:1026C00013F00401430E826F6DEC0EF06DEF13F00A
:1026D0000401630E826F6DEC0EF011A277EF13F020
:1026E0000401500E826F6DEC0EF07CEF13F00401CC
:1026F000700E826F6DEC0EF011A486EF13F00401E2
:10270000550E826F6DEC0EF08BEF13F00401750E19
:10271000826F6DEC0EF00DEF26F004016D0E826FEE
:102720006DEC0EF003018351300AD8B4E5EF13F0DD
:1027300003018351310AD8B4F8EF13F00301835138
:10274000320AD8B40BEF14F00FEF26F004014D0E4F
:10275000826F6DEC0EF010EC2DF084C331F185C367
:1027600032F186C333F10101296B1DEC2DF094EC9D
:102770002CF003018351300AD8B4CDEF13F00301DC
:102780008351310AD8B4D5EF13F003018351320AD3
:10279000D8B4DDEF13F00FEF26F0FD0E0C6E00C184
:1027A0000BF002EC0BF0E5EF13F0FE0E0C6E00C127
:1027B0000BF002EC0BF0F8EF13F0FF0E0C6E00C103
:1027C0000BF002EC0BF00BEF14F00401300E826FF3
:1027D0006DEC0EF004012C0E826F6DEC0EF0CFEC60
:1027E0002CF0FD0E19EC0BF0E8CF00F11CEF14F00B
:1027F0000401310E826F6DEC0EF004012C0E826F1D
:102800006DEC0EF0CFEC2CF0FE0E19EC0BF0E8CFD7
:1028100000F11CEF14F00401320E826F6DEC0EF02B
:10282000CFEC2CF004012C0E826F6DEC0EF0FF0E3D
:1028300019EC0BF0E8CF00F172EC2CF031C182F40E
:102840000401300E82276DEC0EF032C182F40401D7
:10285000300E82276DEC0EF033C182F40401300E8D
:1028600082276DEC0EF00DEF26F003018351300A44
:10287000D8B430EF19F003018351310AD8B45DEFB9
:102880001AF003018351320AD8B4CBEF1AF00301D6
:102890008351330AD8B4DBEF1AF003018351340AB1
:1028A000D8B4EBEF1AF003018351350AD8B45CEFCA
:1028B0001CF003018351360AD8B48AEF1CF00301DF
:1028C0008351370AD8B408EF17F003018351380A4F
:1028D000D8B4A6EF17F003018351460AD8B4B0EF7D
:1028E0001BF0030183514D0AD8B481EF15F00301A9
:1028F00083516D0AD8B49BEF15F0030183515A0A36
:10290000D8B4D7EF19F003018351490AD8B48AEF3C
:102910001DF003018351500AD8B4BCEF1CF0030131
:102920008351540AD8B435EF1DF003018351630A73
:10293000D8B4BBEF15F003018351430AD8B4B3EF09
:1029400016F003018351730AD8B4B9EF15F00301EF
:102950008351610AD8B4CEEF14F003018351650AA4
:10296000D8B480EF19F003018351450AD8B48EEF33
:1029700019F003018351620AD8B49CEF19F00301E6
:102980008351420AD8B4AAEF19F003018351760AA1
:10299000D8B4B8EF19F0D8A40FEF26F004014C0E0C
:1029A000826F6DEC0EF00401610E826F6DEC0EF023
:1029B000FFEC2DF004012C0E826F6DEC0EF0CFECCD
:1029C0002CF0AFC500F1010172EC2CF031C182F4A2
:1029D0000401300E82276DEC0EF032C182F4040146
:1029E000300E82276DEC0EF033C182F40401300EFC
:1029F00082276DEC0EF004012C0E826F6DEC0EF050
:102A0000CFEC2CF0B0C500F1010172EC2CF031C11B
:102A100082F40401300E82276DEC0EF032C182F494
:102A20000401300E82276DEC0EF033C182F40401F4
:102A3000300E82276DEC0EF004012C0E826F6DECCF
:102A40000EF0CFEC2CF0B1C500F1010172EC2CF0CE
:102A500031C182F40401300E82276DEC0EF032C1D8
:102A600082F40401300E82276DEC0EF033C182F443
:102A70000401300E82276DEC0EF004012C0E826FE3
:102A80006DEC0EF0CFEC2CF0B2C500F1010172EC50
:102A90002CF031C182F40401300E82276DEC0EF06F
:102AA00032C182F40401300E82276DEC0EF033C186
:102AB00082F40401300E82276DEC0EF004012C0E1E
:102AC000826F6DEC0EF0CFEC2CF0B6C500F1010179
:102AD00072EC2CF031C182F40401300E82276DECCF
:102AE0000EF032C182F40401300E82276DEC0EF03C
:102AF00033C182F40401300E82276DEC0EF0B8EF82
:102B00001CF010EC2DF084C333F11DEC2DF094EC8F
:102B10002CF0200E0C6E00C10BF002EC0BF000C18B
:102B20002FF505012F51000A06E005012F51010A7A
:102B300002E099EC2EF004014C0E826F6DEC0EF069
:102B400004014D0E826F6DEC0EF004012C0E826FAD
:102B50006DEC0EF0CFEC2CF02FC500F172EC2CF0E8
:102B600033C182F40401300E82276DEC0EF0B8EF11
:102B70001CF071EF33F004014C0E826F6DEC0EF01F
:102B80000401630E826F6DEC0EF057EC2DF0040122
:102B90002C0E826F6DEC0EF0D0EC15F0B8EF1CF03F
:102BA000CFEC2CF0B5C500F10101003B0F0E001772
:102BB00072EC2CF033C182F40401300E82276DECEC
:102BC0000EF0B5C500F101010F0E0101001772EC06
:102BD0002CF033C182F40401300E82276DEC0EF02C
:102BE00004012D0E826F6DEC0EF0B4C500F10101F1
:102BF000003B0F0E001772EC2CF033C182F404017D
:102C0000300E82276DEC0EF0B4C500F101010F0EFD
:102C10000101001772EC2CF033C182F40401300E74
:102C200082276DEC0EF004012D0E826F6DEC0EF01C
:102C3000B3C500F10101003B0F0E001772EC2CF040
:102C400033C182F40401300E82276DEC0EF0B3C55F
:102C500000F101010F0E0101001772EC2CF033C1DD
:102C600082F40401300E82276DEC0EF00401200E78
:102C7000826F6DEC0EF0B2C500F10F0E010100176E
:102C800072EC2CF033C182F40401300E82276DEC1B
:102C90000EF00401200E826F6DEC0EF0B1C500F154
:102CA00001010101003B0F0E001772EC2CF033C143
:102CB00082F40401300E82276DEC0EF0B1C500F1F4
:102CC00001010F0E0101001772EC2CF033C182F4E8
:102CD0000401300E82276DEC0EF004013A0E826F73
:102CE0006DEC0EF0B0C500F10101003B0F0E0017B6
:102CF00072EC2CF033C182F40401300E82276DECAB
:102D00000EF0B0C500F101010F0E0101001772ECC9
:102D10002CF033C182F40401300E82276DEC0EF0EA
:102D200004013A0E826F6DEC0EF0AFC500F10101A7
:102D3000003B0F0E001772EC2CF033C182F404013B
:102D4000300E82276DEC0EF0AFC500F101010F0EC1
:102D5000001772EC2CF033C182F40401300E82278C
:102D60006DEC0EF0120084C3E8FF0F0BE83AE8CFD9
:102D7000B5F585C3E8FF0F0B0501B51387C3E8FF61
:102D80000F0BE83AE8CFB4F588C3E8FF0F0B050155
:102D9000B4138AC3E8FF0F0BE83AE8CFB3F58BC34F
:102DA000E8FF0F0B0501B3138DC3E8FF0F0BE8CF4E
:102DB000B2F58FC3E8FF0F0BE83AE8CFB1F590C347
:102DC000E8FF0F0B0501B11392C3E8FF0F0BE83AC0
:102DD000E8CFB0F593C3E8FF0F0B0501B01395C31F
:102DE000E8FF0F0BE83AE8CFAFF596C3E8FF0F0B0B
:102DF0000501AF13B2EC2DF004014C0E826F6DECA7
:102E00000EF00401430E826F6DEC0EF0C5EF15F06D
:102E1000078404014C0E826F6DEC0EF00401370E36
:102E2000826F6DEC0EF004012C0E826F6DEC0EF0D3
:102E300005012E51130A06E005012E51170A0DE077
:102E4000A3EF17F00101000E006F000E016F100ECE
:102E5000026F000E036F36EF17F00101000E006FD6
:102E6000000E016F000E026F010E036F72EC2CF06A
:102E70002AC182F40401300E82276DEC0EF02BC1C2
:102E800082F40401300E82276DEC0EF02CC182F426
:102E90000401300E82276DEC0EF02DC182F4040186
:102EA000300E82276DEC0EF02EC182F40401300E3C
:102EB00082276DEC0EF02FC182F40401300E8227C0
:102EC0006DEC0EF030C182F40401300E82276DECFF
:102ED0000EF031C182F40401300E82276DEC0EF049
:102EE00032C182F40401300E82276DEC0EF033C142
:102EF00082F40401300E82276DEC0EF004012C0EDA
:102F0000826F6DEC0EF00101100E006F000E016F6C
:102F1000000E026F000E036F72EC2CF031C182F4D0
:102F20000401300E82276DEC0EF032C182F40401F0
:102F3000300E82276DEC0EF033C182F40401300EA6
:102F400082276DEC0EF00794B8EF1CF00501216BA1
:102F5000226B236B246B04014C0E826F6DEC0EF020
:102F60000401380E826F6DEC0EF004012C0E826F9E
:102F70006DEC0EF00101100E006F000E016F000EDF
:102F8000026F000E036F72EC2CF02AC182F4040170
:102F9000300E82276DEC0EF02BC182F40401300E4E
:102FA00082276DEC0EF02CC182F40401300E8227D2
:102FB0006DEC0EF02DC182F40401300E82276DEC11
:102FC0000EF02EC182F40401300E82276DEC0EF05B
:102FD0002FC182F40401300E82276DEC0EF030C157
:102FE00082F40401300E82276DEC0EF031C182F4C0
:102FF0000401300E82276DEC0EF032C182F4040120
:10300000300E82276DEC0EF033C182F40401300ED5
:1030100082276DEC0EF004012C0E826F6DEC0EF029
:1030200025C500F126C501F127C502F128C503F128
:103030000101100E046F000E056F000E066F000EEA
:10304000076F05EC2CF000C133F501C134F502C166
:1030500035F503C136F572EC2CF02AC182F4040177
:10306000300E82276DEC0EF02BC182F40401300E7D
:1030700082276DEC0EF02CC182F40401300E822701
:103080006DEC0EF02DC182F40401300E82276DEC40
:103090000EF02EC182F40401300E82276DEC0EF08A
:1030A0002FC182F40401300E82276DEC0EF030C186
:1030B00082F40401300E82276DEC0EF031C182F4EF
:1030C0000401300E82276DEC0EF032C182F404014F
:1030D000300E82276DEC0EF033C182F40401300E05
:1030E00082276DEC0EF077EC0EF00501336780EF70
:1030F00018F0346780EF18F0356780EF18F0366706
:1031000002D01FEF19F0129E129C21C500F122C5BA
:1031100001F123C502F124C503F1899A400EC76E5F
:10312000200EC66E9E96C69E0B0EC96EFF0E9EB6F4
:1031300002D0E82EFCD79E96C69E02C1C9FFFF0EA4
:103140009EB602D0E82EFCD79E96C69E01C1C9FF4E
:10315000FF0E9EB602D0E82EFCD79E96C69E00C1FA
:10316000C9FFFF0E9EB602D0E82EFCD79E96C69EE3
:10317000C952FF0E9EB602D0E82EFCD70501100EF4
:10318000326F040114EE00F080517F0BE1269E9611
:10319000C69EC952FF0E9EB602D0E82EFCD7C9CFFC
:1031A000E7FF0401802B0501322FC1EF18F0898A57
:1031B00033C500F134C501F135C502F136C503F15F
:1031C0000101010E046F000E056F000E066F000E68
:1031D000076FD4EC2BF000C133F501C134F502C107
:1031E00035F503C136F505013367FEEF18F0346796
:1031F000FEEF18F03567FEEF18F0366702D01FEFCC
:1032000019F021C500F122C501F123C502F124C541
:1032100003F10101100E046F000E056F000E066F22
:10322000000E076FD9EC2BF000C121F501C122F58A
:1032300002C123F503C124F5128E0FEF26F004011D
:10324000450E826F6DEC0EF004014F0E826F6DEC37
:103250000EF00401460E826F6DEC0EF0B8EF1CF01C
:10326000078432EC33F0CFEC2CF02DC500F172EC7A
:103270002CF004014C0E826F6DEC0EF00401300E48
:10328000826F6DEC0EF004012C0E826F6DEC0EF06F
:1032900031C182F40401300E82276DEC0EF032C190
:1032A00082F40401300E82276DEC0EF033C182F4FB
:1032B0000401300E82276DEC0EF004012C0E826F9B
:1032C0006DEC0EF0CFEC2CF02EC500F172EC2CF072
:1032D00031C182F40401300E82276DEC0EF032C150
:1032E00082F40401300E82276DEC0EF033C182F4BB
:1032F0000401300E82276DEC0EF00794B8EF1CF03D
:1033000004014C0E826F6DEC0EF00401650E826FAD
:103310006DEC0EF059EC2FF0B8EF1CF004014C0EE0
:10332000826F6DEC0EF00401450E826F6DEC0EF0B5
:1033300070EC2FF0B8EF1CF004014C0E826F6DECB6
:103340000EF00401620E826F6DEC0EF09EEC2FF019
:10335000B8EF1CF004014C0E826F6DEC0EF004010E
:10336000420E826F6DEC0EF087EC2FF0B8EF1CF080
:1033700004014C0E826F6DEC0EF00401760E826F2C
:103380006DEC0EF004012C0E826F6DEC0EF010A8A7
:1033900007D00401310E826F6DEC0EF0B8EF1CF017
:1033A0000401300E826F6DEC0EF0B8EF1CF00401DA
:1033B0004C0E826F6DEC0EF004015A0E826F6DECB4
:1033C0000EF004012C0E826F6DEC0EF032EC33F037
:1033D000CFEC2CF005012E51130A06E005012E5109
:1033E000170A0DE008EF1AF00101000E006F000E41
:1033F000016F100E026F000E036F08EF1AF001014B
:10340000000E006F000E016F000E026F010E036FC1
:103410000101100E046F000E056F000E066F000E06
:10342000076F05EC2CF072EC2CF02AC182F4040139
:10343000300E82276DEC0EF02BC182F40401300EA9
:1034400082276DEC0EF02CC182F40401300E82272D
:103450006DEC0EF02DC182F40401300E82276DEC6C
:103460000EF02EC182F40401300E82276DEC0EF0B6
:103470002FC182F40401300E82276DEC0EF030C1B2
:1034800082F40401300E82276DEC0EF031C182F41B
:103490000401300E82276DEC0EF032C182F404017B
:1034A000300E82276DEC0EF033C182F40401300E31
:1034B00082276DEC0EF0B8EF1CF0078404014C0E6F
:1034C000826F6DEC0EF00401310E826F6DEC0EF028
:1034D00004012C0E826F6DEC0EF025C500F126C59F
:1034E00001F127C502F128C503F10101100E046F97
:1034F000000E056F000E066F000E076F05EC2CF036
:1035000072EC2CF02AC182F40401300E82276DEC9B
:103510000EF02BC182F40401300E82276DEC0EF008
:103520002CC182F40401300E82276DEC0EF02DC107
:1035300082F40401300E82276DEC0EF02EC182F46D
:103540000401300E82276DEC0EF02FC182F40401CD
:10355000300E82276DEC0EF030C182F40401300E83
:1035600082276DEC0EF031C182F40401300E822707
:103570006DEC0EF032C182F40401300E82276DEC46
:103580000EF033C182F40401300E82276DEC0EF090
:103590000794B8EF1CF0078404014C0E826F6DECA9
:1035A0000EF00401320E826F6DEC0EF08CEC31F0F7
:1035B0000794B8EF1CF0078404014C0E826F6DEC89
:1035C0000EF00401330E826F6DEC0EF0E9EC31F079
:1035D000079468EF1AF0078404014C0E826F6DECBB
:1035E0000EF00401340E826F6DEC0EF004012C0E0F
:1035F000826F6DEC0EF010EC2DF084C32AF185C3C0
:103600002BF186C32CF187C32DF188C32EF189C31A
:103610002FF18AC330F18BC331F18CC332F18DC3EA
:1036200033F10101296B1DEC2DF094EC2CF0100E00
:10363000046F000E056F000E066F000E076FE5ECBD
:103640002BF000C121F501C122F502C123F503C110
:1036500024F5E5EC32F038C5AFF539C5B0F53AC51B
:10366000B1F53BC5B2F53CC5B3F53DC5B4F53EC5B6
:10367000B5F5D0EC15F004012C0E826F6DEC0EF058
:103680003FC500F140C501F141C502F142C503F15A
:103690000101000E046F000E056F010E066F000E93
:1036A000076F05EC2CF072EC2CF029675AEF1BF039
:1036B0005FEF1BF004012D0E826F6DEC0EF030C138
:1036C00082F40401300E82276DEC0EF031C182F4D9
:1036D0000401300E82276DEC0EF004012E0E826F75
:1036E0006DEC0EF032C182F40401300E82276DECD5
:1036F0000EF033C182F40401300E82276DEC0EF01F
:1037000004012C0E826F6DEC0EF0CFEC2CF043C553
:1037100000F144C501F139EC27F004012C0E826F51
:103720006DEC0EF0CFEC2CF045C500F172EC2CF0F6
:1037300031C182F40401300E82276DEC0EF032C1EB
:1037400082F40401300E82276DEC0EF033C182F456
:103750000401300E82276DEC0EF00794B8EF1CF0D8
:1037600010EC2DF085C32AF186C32BF187C32CF111
:1037700088C32DF189C32EF18AC32FF18BC330F199
:103780008CC331F18DC332F18EC333F10101296B4A
:103790001DEC2DF094EC2CF00101010E046F000ED5
:1037A000056F000E066F000E076FD4EC2BF0100EA5
:1037B000046F000E056F000E066F000E076FE5EC3C
:1037C0002BF000C129F501C12AF502C12BF503C177
:1037D0002CF513EC31F004014C0E826F6DEC0EF001
:1037E0000401460E826F6DEC0EF004012C0E826F08
:1037F0006DEC0EF025C500F126C501F127C502F1DB
:1038000028C503F10101100E046F000E056F000EB4
:10381000066F000E076F05EC2CF072EC2CF02AC13D
:1038200082F40401300E82276DEC0EF02BC182F47D
:103830000401300E82276DEC0EF02CC182F40401DD
:10384000300E82276DEC0EF02DC182F40401300E93
:1038500082276DEC0EF02EC182F40401300E822717
:103860006DEC0EF02FC182F40401300E82276DEC56
:103870000EF030C182F40401300E82276DEC0EF0A0
:1038800031C182F40401300E82276DEC0EF032C19A
:1038900082F40401300E82276DEC0EF033C182F405
:1038A0000401300E82276DEC0EF0B8EF1CF00F987B
:1038B000E9EC31F00FEF26F004014C0E826F6DEC55
:1038C0000EF00401350E826F6DEC0EF004012C0E2B
:1038D000826F6DEC0EF0CFEC2CF00784B9C500F1CF
:1038E000079472EC2CF031C182F40401300E82276F
:1038F0006DEC0EF032C182F40401300E82276DECC3
:103900000EF033C182F40401300E82276DEC0EF00C
:10391000B8EF1CF0ACEC31F0CFEC2CF037C500F177
:1039200072EC2CF004014C0E826F6DEC0EF0040171
:10393000360E826F6DEC0EF004012C0E826F6DEC72
:103940000EF031C182F40401300E82276DEC0EF0CE
:1039500032C182F40401300E82276DEC0EF033C1C7
:1039600082F40401300E82276DEC0EF0B8EF1CF0EB
:1039700077EC0EF00FEF26F004014C0E826F6DEC29
:103980000EF00401500E826F6DEC0EF004012C0E4F
:10399000826F6DEC0EF085C32AF186C32BF187C3CD
:1039A0002CF188C32DF189C32EF18AC32FF18BC36B
:1039B00030F18CC331F18DC332F18EC333F101018B
:1039C0001DEC2DF094EC2CF003018451530A0DE012
:1039D000030184514D0A38E00401780E826F6DECCA
:1039E0000EF077EC0EF00FEF26F00401530E826F0D
:1039F0006DEC0EF0250E0C6E00C10BF002EC0BF01E
:103A0000260E0C6E01C10BF002EC0BF0270E0C6EB3
:103A100002C10BF002EC0BF0280E0C6E03C10BF090
:103A200002EC0BF000C157F501C158F502C159F580
:103A300003C15AF500C15BF501C15CF502C15DF53A
:103A400003C15EF599EF1DF004014D0E826F6DEC20
:103A50000EF0290E0C6E00C10BF002EC0BF000C151
:103A60005FF500C160F599EF1DF004014C0E826F07
:103A70006DEC0EF00401540E826F6DEC0EF004013B
:103A80002C0E826F6DEC0EF084C32AF185C32BF1EE
:103A900086C32CF187C32DF188C32EF189C32FF182
:103AA0008AC330F18BC331F18DC332F18EC333F150
:103AB00001011DEC2DF094EC2CF00101000E046FBF
:103AC000000E056F010E066F000E076FE5EC2BF080
:103AD000210E0C6E00C10BF002EC0BF0220E0C6EEE
:103AE00001C10BF002EC0BF0230E0C6E02C10BF0C7
:103AF00002EC0BF0240E0C6E03C10BF002EC0BF089
:103B000000C161F501C162F502C163F503C164F54D
:103B100099EF1DF004014C0E826F6DEC0EF0040164
:103B2000490E826F6DEC0EF004012C0E826F6DEC6D
:103B30000EF0250E19EC0BF0E8CF00F1260E19EC73
:103B40000BF0E8CF01F1270E19EC0BF0E8CF02F1F2
:103B5000280E19EC0BF0E8CF03F172EC2CF055ECC9
:103B60002AF00401730E826F6DEC0EF004012C0E2E
:103B7000826F6DEC0EF0CFEC2CF0290E19EC0BF0EF
:103B8000E8CF00F172EC2CF055EC2AF00401730E32
:103B9000826F6DEC0EF004012C0E826F6DEC0EF056
:103BA0005BC500F15CC501F15DC502F15EC503F1C5
:103BB00072EC2CF055EC2AF00401730E826F6DEC60
:103BC0000EF004012C0E826F6DEC0EF0CFEC2CF099
:103BD00060C500F172EC2CF055EC2AF004016D0E7A
:103BE000826F6DEC0EF004012C0E826F6DEC0EF006
:103BF00061C500F162C501F163C502F164C503F15D
:103C00002AEC26F004012C0E826F6DEC0EF077EC9E
:103C10000EF00FEF26F083C32AF184C32BF185C386
:103C20002CF186C32DF187C32EF188C32FF189C3F0
:103C300030F18AC331F18BC332F18CC333F101010E
:103C40001DEC2DF094EC2CF0160E0C6E00C10BF058
:103C500002EC0BF0170E0C6E01C10BF002EC0BF036
:103C6000180E0C6E02C10BF002EC0BF0190E0C6E6C
:103C700003C10BF002EC0BF000C18AF101C18BF122
:103C800002C18CF103C18DF100C18EF101C18FF130
:103C900002C190F103C191F1EDEF1EF083C32AF14F
:103CA00084C32BF185C32CF186C32DF187C32EF17C
:103CB00088C32FF189C330F18AC331F18BC332F14C
:103CC0008CC333F101011DEC2DF094EC2CF000C1FC
:103CD0008AF101C18BF102C18CF103C18DF100C1E8
:103CE0008EF101C18FF102C190F103C191F1EDEFAD
:103CF0001EF083C32AF184C32BF185C32CF186C344
:103D00002DF187C32EF188C32FF189C330F18AC307
:103D100031F18CC332F18DC333F101011DEC2DF073
:103D200094EC2CF00101000E046F000E056F010EE3
:103D3000066F000E076FE5EC2BF01A0E0C6E00C13B
:103D40000BF002EC0BF01B0E0C6E01C10BF002EC41
:103D50000BF01C0E0C6E02C10BF002EC0BF01D0EF2
:103D60000C6E03C10BF002EC0BF000C192F101C12B
:103D700093F102C194F103C195F1EDEF1EF083C3FD
:103D80002AF184C32BF185C32CF186C32DF187C39F
:103D90002EF188C32FF189C330F18AC331F18CC36E
:103DA00032F18DC333F101011DEC2DF094EC2CF0B8
:103DB0000101000E046F000E056F010E066F000E6C
:103DC000076FE5EC2BF000C192F101C193F102C144
:103DD00094F103C195F1EDEF1EF0160E19EC0BF006
:103DE000E8CF00F1170E19EC0BF0E8CF01F1180E37
:103DF00019EC0BF0E8CF02F1190E19EC0BF0E8CF3B
:103E000003F172EC2CF055EC2AF00401730E826F72
:103E10006DEC0EF004012C0E826F6DEC0EF08AC179
:103E200000F18BC101F18CC102F18DC103F172EC83
:103E30002CF055EC2AF00401730E826F6DEC0EF03D
:103E400004012C0E826F6DEC0EF01A0E19EC0BF0C3
:103E5000E8CF00F11B0E19EC0BF0E8CF01F11C0EBE
:103E600019EC0BF0E8CF02F11D0E19EC0BF0E8CFC6
:103E700003F12AEC26F004012C0E826F6DEC0EF09B
:103E800092C100F193C101F194C102F195C103F116
:103E90002AEC26F077EC0EF00FEF26F00401690E05
:103EA000826F6DEC0EF004012C0E826F6DEC0EF043
:103EB0000101040E006F000E016F000E026F000E74
:103EC000036F72EC2CF02CC182F40401300E8227B7
:103ED0006DEC0EF02DC182F40401300E82276DECE2
:103EE0000EF02EC182F40401300E82276DEC0EF02C
:103EF0002FC182F40401300E82276DEC0EF030C128
:103F000082F40401300E82276DEC0EF031C182F490
:103F10000401300E82276DEC0EF032C182F40401F0
:103F2000300E82276DEC0EF033C182F40401300EA6
:103F300082276DEC0EF004012C0E826F6DEC0EF0FA
:103F40000101060E006F000E016F000E026F000EE1
:103F5000036F72EC2CF02CC182F40401300E822726
:103F60006DEC0EF02DC182F40401300E82276DEC51
:103F70000EF02EC182F40401300E82276DEC0EF09B
:103F80002FC182F40401300E82276DEC0EF030C197
:103F900082F40401300E82276DEC0EF031C182F400
:103FA0000401300E82276DEC0EF032C182F4040160
:103FB000300E82276DEC0EF033C182F40401300E16
:103FC00082276DEC0EF004012C0E826F6DEC0EF06A
:103FD00001012F0E006F000E016F000E026F000E28
:103FE000036F72EC2CF02CC182F40401300E822796
:103FF0006DEC0EF02DC182F40401300E82276DECC1
:104000000EF02EC182F40401300E82276DEC0EF00A
:104010002FC182F40401300E82276DEC0EF030C106
:1040200082F40401300E82276DEC0EF031C182F46F
:104030000401300E82276DEC0EF032C182F40401CF
:10404000300E82276DEC0EF033C182F40401300E85
:1040500082276DEC0EF004012C0E826F6DEC0EF0D9
:10406000200EF86EF76AF66A04010900F5CF82F4B3
:104070006DEC0EF00900F5CF82F46DEC0EF0090046
:10408000F5CF82F46DEC0EF00900F5CF82F46DEC03
:104090000EF00900F5CF82F46DEC0EF00900F5CFBB
:1040A00082F46DEC0EF00900F5CF82F46DEC0EF0A9
:1040B0000900F5CF82F46DEC0EF077EC0EF00FEF07
:1040C00026F08351630AD8A40DEF26F08451610ACB
:1040D000D8A40DEF26F085516C0AD8A40DEF26F078
:1040E0008651410A3FE08651440A1BE08651420A4C
:1040F000D8B4C5EF20F08651350AD8B499EF27F02F
:104100008651360AD8B4EEEF27F08651370AD8B474
:1041100057EF28F08651380AD8B4B5EF28F00DEFE4
:1041200026F00798079A04017A0E826F6DEC0EF064
:104130000401780E826F6DEC0EF00401640E826F44
:104140006DEC0EF00401550E826F6DEC0EF0AEEFCB
:1041500020F004014C0E826F6DEC0EF077EC0EF047
:104160000FEF26F00788079A04017A0E826F6DEC34
:104170000EF00401410E826F6DEC0EF00401610E31
:10418000826F6DEC0EF0A2EF20F00798078A040111
:104190007A0E826F6DEC0EF00401420E826F6DECB0
:1041A0000EF00401610E826F6DEC0EF0A2EF20F0B4
:1041B00001016667E3EF20F06767E3EF20F06867CF
:1041C000E3EF20F0696715D04F67EEEF20F05067FE
:1041D000EEEF20F05167EEEF20F052670AD00101B8
:1041E000000E006F000E016F000E026F000E036FD5
:1041F000120011B80AD00101620E046F010E056FA2
:10420000000E066F000E076F09D00101A70E046FA4
:10421000020E056F000E066F000E076F66C100F1FB
:1042200067C101F168C102F169C103F1D4EC2BF05F
:1042300003BF8BEF21F0119A119C0101000E046F56
:10424000A80E056F550E066F020E076F66C100F1CE
:1042500067C101F168C102F169C103F166C186F16C
:1042600067C187F168C188F169C189F1D4EC2BF08D
:1042700003BF0BD00101000E866FA80E876F550E8D
:10428000886F020E896F118A119C0E0E19EC0BF0CB
:10429000E8CF18F10F0E19EC0BF0E8CF19F1100E62
:1042A00019EC0BF0E8CF1AF1110E19EC0BF0E8CF76
:1042B0001BF11DEC2BF086C104F187C105F188C10B
:1042C00006F189C107F1D4EC2BF00782E1EC2AF06A
:1042D0001DEC2BF00792E1EC2AF086C100F187C1BA
:1042E00001F188C102F189C103F10792E1EC2AF0E2
:1042F000CC0E046FE00E056F870E066F050E076F7C
:10430000D4EC2BF000C118F101C119F102C11AF16E
:1043100003C11BF13BD0119C119A0101800E006F6B
:104320001A0E016F060E026F000E036F4FC104F1EB
:1043300050C105F151C106F152C107F1D4EC2BF087
:1043400003AF05D0CFEC2CF0118C119A12000E0E99
:1043500019EC0BF0E8CF18F10F0E19EC0BF0E8CFC9
:1043600019F1100E19EC0BF0E8CF1AF1110E19EC3F
:104370000BF0E8CF1BF14FC100F150C101F151C169
:1043800002F152C103F10782E1EC2AF018C100F1F9
:1043900019C101F11AC102F11BC103F1120004019C
:1043A000730E826F6DEC0EF004012C0E826F6DECBB
:1043B0000EF0078462C166F163C167F164C168F100
:1043C00065C169F14BC14FF14CC150F14DC151F183
:1043D0004EC152F157C159F158C15AF10794F5EC49
:1043E00021F077EC0EF00FEF26F066C100F167C107
:1043F00001F168C102F169C103F1010172EC2CF015
:1044000055EC2AF00401630E826F6DEC0EF004018E
:104410002C0E826F6DEC0EF04FC100F150C101F116
:1044200051C102F152C103F1010172EC2CF055ECC3
:104430002AF00401660E826F6DEC0EF004012C0E62
:10444000826F6DEC0EF0CFEC2CF059C100F15AC127
:1044500001F1010172EC2CF055EC2AF00401740E0C
:10446000826F6DEC0EF0120010820401530E826F09
:104470006DEC0EF004012C0E826F6DEC0EF083C318
:104480002AF184C32BF185C32CF186C32DF187C398
:104490002EF188C32FF189C330F18AC331F18BC368
:1044A00032F18CC333F101011DEC2DF094EC2CF0B2
:1044B00000C166F101C167F102C168F103C169F190
:1044C0008EC32AF18FC32BF190C32CF191C32DF130
:1044D00092C32EF193C32FF194C330F195C331F100
:1044E00096C332F197C333F101011DEC2DF094EC2A
:1044F0002CF000C14FF101C150F102C151F103C1D3
:1045000052F110EC2DF099C32FF19AC330F19BC3F7
:1045100031F19CC332F19DC333F101011DEC2DF04B
:1045200094EC2CF000C159F101C15AF1F5EC21F0E5
:1045300004012C0E826F6DEC0EF0AEEF22F0118EA6
:1045400018A002D018AE108C17BE02D017A4108E7F
:104550008251520A02E10F8201D00F928251750AF4
:1045600002E1108401D010948251550A02E11086B4
:1045700001D0109611A003D011A401D0108407849B
:1045800010B21CEF23F010A408EF23F0B6C166F1BF
:10459000B7C167F1B8C168F1B9C169F1BAC16AF1CF
:1045A000BBC16BF1BCC16CF1BDC16DF1BEC16EF19F
:1045B000BFC16FF1C0C170F1C1C171F1C2C172F16F
:1045C000C3C173F1C4C174F1C5C175F1C6C176F13F
:1045D000C7C177F1C8C178F1C9C179F1CAC17AF10F
:1045E000CBC17BF1CCC17CF1CDC17DF1CEC17EF1DF
:1045F000CFC17FF1D0C180F1D1C181F1D2C182F1AF
:10460000D3C183F1D4C184F1D5C185F110EF23F07A
:1046100062C166F163C167F164C168F165C169F1A6
:104620004BC14FF14CC150F14DC151F14EC152F14E
:1046300057C159F158C15AF107940FA03EEF23F02A
:10464000010192672BEF23F093672BEF23F0946720
:104650002BEF23F095672FEF23F03EEF23F0D8ECFC
:1046600020F092C104F193C105F194C106F195C106
:1046700007F1D4EC2BF003BFD5EF25F0D8EC20F0F8
:104680000101000E046F000E056F010E066F000E93
:10469000076F05EC2CF011A02CD011A22AD072ECDF
:1046A0002CF0296701D007D004012D0E826F6DEC2C
:1046B0000EF0D3EF25F030C182F40401300E8227D2
:1046C0006DEC0EF031C182F40401300E82276DECE6
:1046D0000EF032C182F40401300E82276DEC0EF030
:1046E00033C182F40401300E82276DEC0EF0D3EF5B
:1046F00025F012A8C5D0129819C01AF01A3A1A4219
:10470000070E1A1600011A50000AD8B40CEF24F054
:1047100000011A50010AD8B498EF23F000011A5092
:10472000020AD8B496EF23F03EEF24F03EEF24F0D7
:10473000CFEC2CF029C001F12AC000F1D890013350
:104740000033D890013300330101630E046F000E73
:10475000056F000E066F000E076F05EC2CF0280E9B
:10476000046F000E056F000E066F000E076FD4EC8D
:104770002BF000C12CF0CFEC2CF027C001F1019FF1
:10478000019D28C000F10101A40E046F000E056F09
:10479000000E066F000E076F05EC2CF000C12BF029
:1047A00000C104F101C105F102C106F103C107F125
:1047B000640E006F000E016F000E026F000E036F9B
:1047C000D4EC2BF0050E046F000E056F000E066F83
:1047D000000E076F05EC2CF000C104F101C105F1DA
:1047E00002C106F103C107F1CFEC2CF02CC000F19F
:1047F000D4EC2BF000C12DF02DC0E8FF050F2C5C90
:1048000003E78A843EEF24F02DC0E8FF0A0F2C5CFA
:1048100001E68A943EEF24F000C124F101C125F1A4
:1048200002C126F103C127F1CFEC2CF0D5EC2CF01E
:1048300019501F0BE8CF00F10101640E046F000E48
:10484000056F000E066F000E076FE5EC2BF024C11C
:1048500004F125C105F126C106F127C107F1D4EC09
:104860002BF003BF02D08A9401D08A8424C100F1C6
:1048700025C101F126C102F127C103F1D5EF25F0D1
:1048800000C124F101C125F102C126F103C127F1C4
:1048900010AE4CD0109E00C108F101C109F102C157
:1048A0000AF103C10BF172EC2CF030C1D6F131C129
:1048B000D7F132C1D8F133C1D9F108C100F109C132
:1048C00001F10AC102F10BC103F101016C0E046F89
:1048D000070E056F000E066F000E076FD4EC2BF06D
:1048E00003BF04D00101550EDA6F1CD008C100F1DE
:1048F00009C101F10AC102F10BC103F10101A40ECA
:10490000046F060E056F000E066F000E076FD4ECE5
:104910002BF003BF04D001017F0EDA6F03D0010139
:10492000FF0EDA6F1B8E11AED5EF25F024C100F11A
:1049300025C101F126C102F127C103F110A4A8EF9E
:1049400024F00401750E826F6DEC0EF0ADEF24F0D3
:104950000401720E826F6DEC0EF004012C0E826F5A
:104960006DEC0EF072EC2CF02967BCEF24F0040122
:10497000200E826FBFEF24F004012D0E826F6DECCC
:104980000EF030C182F40401300E82276DEC0EF07F
:1049900031C182F40401300E82276DEC0EF0040167
:1049A0002E0E826F6DEC0EF032C182F40401300ED7
:1049B00082276DEC0EF033C182F40401300E8227A1
:1049C0006DEC0EF004016D0E826F6DEC0EF00401C3
:1049D0002C0E826F6DEC0EF04FC100F150C101F151
:1049E00051C102F152C103F1010172EC2CF055ECFE
:1049F0002AF00401480E826F6DEC0EF004017A0E6D
:104A0000826F6DEC0EF004012C0E826F6DEC0EF0D7
:104A100066C100F167C101F168C102F169C103F12A
:104A2000010172EC2CF055EC2AF00401630E826F48
:104A30006DEC0EF004012C0E826F6DEC0EF066C171
:104A400000F167C101F168C102F169C103F101011F
:104A50000A0E046F000E056F000E066F000E076F42
:104A6000E5EC2BF0000E046F120E056F000E066FC2
:104A7000000E076F05EC2CF072EC2CF02AC182F4CA
:104A80000401300E82276DEC0EF02BC182F404017C
:104A9000300E82276DEC0EF02CC182F40401300E32
:104AA00082276DEC0EF02DC182F40401300E8227B6
:104AB0006DEC0EF02EC182F40401300E82276DECF5
:104AC0000EF02FC182F40401300E82276DEC0EF03F
:104AD00030C182F40401300E82276DEC0EF0040127
:104AE0002E0E826F6DEC0EF031C182F40401300E97
:104AF00082276DEC0EF032C182F40401300E822761
:104B00006DEC0EF033C182F40401300E82276DEC9F
:104B10000EF00401730E826F6DEC0EF004012C0E8A
:104B2000826F6DEC0EF0CFEC2CF059C100F15AC140
:104B300001F139EC27F00FB2A1EF25F00FA0D3EF70
:104B400025F004012C0E826F6DEC0EF0200EF86E35
:104B5000F76AF66A04010900F5CF82F46DEC0EF0F5
:104B60000900F5CF82F46DEC0EF00900F5CF82F468
:104B70006DEC0EF00900F5CF82F46DEC0EF009003B
:104B8000F5CF82F46DEC0EF00900F5CF82F46DECF8
:104B90000EF00900F5CF82F46DEC0EF00900F5CFB0
:104BA00082F46DEC0EF077EC0EF00F900FEF26F024
:104BB0000401630E826F6DEC0EF004012C0E826F07
:104BC0006DEC0EF015EC26F004012C0E826F6DECEE
:104BD0000EF088EC26F004012C0E826F6DEC0EF0C6
:104BE00004EC27F004012C0E826F6DEC0EF0010135
:104BF000F80E006FCD0E016F660E026F030E036F8D
:104C00002AEC26F004012C0E826F6DEC0EF01AECEB
:104C100027F077EC0EF00FEF26F077EC0EF00301A3
:104C2000C26B079010921EEF29F0D8900E0E19EC6F
:104C30000BF0E8CF00F10F0E19EC0BF0E8CF01F10B
:104C4000100E19EC0BF0E8CF02F1110E19EC0BF07D
:104C5000E8CF03F10101000E046F000E056F010E95
:104C6000066F000E076F05EC2CF072EC2CF02AC1D9
:104C700082F40401300E82276DEC0EF02BC182F419
:104C80000401300E82276DEC0EF02CC182F4040179
:104C9000300E82276DEC0EF02DC182F40401300E2F
:104CA00082276DEC0EF02EC182F40401300E8227B3
:104CB0006DEC0EF02FC182F40401300E82276DECF2
:104CC0000EF030C182F40401300E82276DEC0EF03C
:104CD00031C182F40401300E82276DEC0EF0040124
:104CE0002E0E826F6DEC0EF032C182F40401300E94
:104CF00082276DEC0EF033C182F40401300E82275E
:104D00006DEC0EF004016D0E826F6DEC0EF0120072
:104D1000120E19EC0BF0E8CF00F1130E19EC0BF0AA
:104D2000E8CF01F1140E19EC0BF0E8CF02F1150EEB
:104D300019EC0BF0E8CF03F101010A0E046F000E2D
:104D4000056F000E066F000E076FE5EC2BF0000EEE
:104D5000046F120E056F000E066F000E076F05EC54
:104D60002CF072EC2CF02AC182F40401300E822760
:104D70006DEC0EF02BC182F40401300E82276DEC35
:104D80000EF02CC182F40401300E82276DEC0EF07F
:104D90002DC182F40401300E82276DEC0EF02EC17D
:104DA00082F40401300E82276DEC0EF02FC182F4E4
:104DB0000401300E82276DEC0EF030C182F4040144
:104DC000300E82276DEC0EF004012E0E826F6DEC1A
:104DD0000EF031C182F40401300E82276DEC0EF02A
:104DE00032C182F40401300E82276DEC0EF033C123
:104DF00082F40401300E82276DEC0EF00401730E74
:104E0000826F6DEC0EF012000A0E19EC0BF0E8CF79
:104E100000F10B0E19EC0BF0E8CF01F10C0E19ECC0
:104E20000BF0E8CF02F10D0E19EC0BF0E8CF03F117
:104E300039EF27F0060E19EC0BF0E8CF00F1070E62
:104E400019EC0BF0E8CF01F1080E19EC0BF0E8CFEC
:104E500002F1090E19EC0BF0E8CF03F139EF27F05E
:104E60000101CFEC2CF0078457C100F158C101F1CA
:104E700007940101E80E046F800E056F000E066FA7
:104E8000000E076FE5EC2BF0000E046F040E056FAB
:104E9000000E066F000E076F05EC2CF0880E046FF5
:104EA000130E056F000E066F000E076FD4EC2BF08B
:104EB0000A0E046F000E056F000E066F000E076FDE
:104EC00005EC2CF072EC2CF0010129676DEF27F056
:104ED0000401200E826F70EF27F004012D0E826F07
:104EE0006DEC0EF030C182F40401300E82276DECBF
:104EF0000EF031C182F40401300E82276DEC0EF009
:104F000032C182F40401300E82276DEC0EF00401F0
:104F10002E0E826F6DEC0EF033C182F40401300E60
:104F200082276DEC0EF00401430E826F6DEC0EF0E3
:104F3000120087C32AF188C32BF189C32CF18AC3DD
:104F40002DF18BC32EF18CC32FF18DC330F18EC3A5
:104F500031F190C332F191C333F10101296B1DECA2
:104F60002DF094EC2CF00101000E046F000E056F83
:104F7000010E066F000E076FE5EC2BF00E0E0C6EA7
:104F800000C10BF002EC0BF00F0E0C6E01C10BF028
:104F900002EC0BF0100E0C6E02C10BF002EC0BF0E9
:104FA000110E0C6E03C10BF002EC0BF004017A0E33
:104FB000826F6DEC0EF004012C0E826F6DEC0EF022
:104FC0000401350E826F6DEC0EF004012C0E826F21
:104FD0006DEC0EF015EC26F0AEEF20F087C32AF151
:104FE00088C32BF189C32CF18AC32DF18BC32EF119
:104FF0008CC32FF18DC330F18EC331F190C332F1E8
:1050000091C333F10101296B1DEC2DF094EC2CF0D0
:10501000880E046F130E056F000E066F000E076FEB
:10502000D9EC2BF0000E046F040E056F000E066F16
:10503000000E076FE5EC2BF00101E80E046F800E07
:10504000056F000E066F000E076F05EC2CF00A0EC0
:105050000C6E00C10BF002EC0BF00B0E0C6E01C1DC
:105060000BF002EC0BF00C0E0C6E02C10BF002EC1C
:105070000BF00D0E0C6E03C10BF002EC0BF00401F3
:105080007A0E826F6DEC0EF004012C0E826F6DECC7
:105090000EF00401360E826F6DEC0EF004012C0E42
:1050A000826F6DEC0EF004EC27F0AEEF20F087C3BA
:1050B0002AF188C32BF189C32CF18AC32DF18BC34C
:1050C0002EF18CC32FF18DC330F18FC331F190C31A
:1050D00032F191C333F101011DEC2DF094EC2CF071
:1050E000000E046F120E056F000E066F000E076FA4
:1050F000E5EC2BF001010A0E046F000E056F000EA7
:10510000066F000E076F05EC2CF0120E0C6E00C13E
:105110000BF002EC0BF0130E0C6E01C10BF002EC65
:105120000BF0140E0C6E02C10BF002EC0BF0150E1E
:105130000C6E03C10BF002EC0BF004017A0E826FCF
:105140006DEC0EF004012C0E826F6DEC0EF004017C
:10515000370E826F6DEC0EF004012C0E826F6DEC39
:105160000EF088EC26F0AEEF20F087C32AF188C35A
:105170002BF189C32CF18AC32DF18BC32EF18CC383
:105180002FF18DC330F18EC331F190C332F191C351
:1051900033F10101296B1DEC2DF094EC2CF0880EFD
:1051A000046F130E056F000E066F000E076FD9EC2B
:1051B0002BF0000E046F040E056F000E066F000E3C
:1051C000076FE5EC2BF00101E80E046F800E056F10
:1051D000000E066F000E076F05EC2CF0060E0C6E2D
:1051E00000C10BF002EC0BF0070E0C6E01C10BF0CE
:1051F00002EC0BF0080E0C6E02C10BF002EC0BF08F
:10520000090E0C6E03C10BF002EC0BF004017A0ED8
:10521000826F6DEC0EF004012C0E826F6DEC0EF0BF
:105220000401380E826F6DEC0EF004012C0E826FBB
:105230006DEC0EF01AEC27F0AEEF20F007A891EF1E
:1052400029F00101800E006F1A0E016F060E026F29
:10525000000E036F4BC104F14CC105F14DC106F1C5
:105260004EC107F1D4EC2BF003BFD7EF29F04FEC80
:105270002AF04BC100F14CC101F14DC102F14EC108
:1052800003F10782E1EC2AF018C104F119C105F11C
:105290001AC106F11BC107F1F80E006FCD0E016FA8
:1052A000660E026F030E036FD4EC2BF00E0E0C6E25
:1052B00000C10BF002EC0BF00F0E0C6E01C10BF0F5
:1052C00002EC0BF0100E0C6E02C10BF002EC0BF0B6
:1052D000110E0C6E03C10BF002EC0BF00784010100
:1052E000CFEC2CF057C100F158C101F107940A0E20
:1052F0000C6E00C10BF002EC0BF00B0E0C6E01C13A
:105300000BF002EC0BF00C0E0C6E02C10BF002EC79
:105310000BF00D0E0C6E03C10BF002EC0BF0D7EF8F
:1053200029F007AAD7EF29F007840101CFEC2CF070
:1053300057C100F158C101F10794060E0C6E00C16F
:105340000BF002EC0BF0070E0C6E01C10BF002EC3F
:105350000BF0080E0C6E02C10BF002EC0BF0090E04
:105360000C6E03C10BF002EC0BF0078462C100F17C
:1053700063C101F164C102F165C103F10794120E2A
:105380000C6E00C10BF002EC0BF0130E0C6E01C1A1
:105390000BF002EC0BF0140E0C6E02C10BF002ECE1
:1053A0000BF0150E0C6E03C10BF002EC0BF007981E
:1053B000079A0401805181197F0B0DE09EA8FED74A
:1053C00014EE00F081517F0BE126E750812B0F0195
:1053D000AD6ED9EF29F005012F51010A13E081AA22
:1053E00002EF2AF005012F51000A0AE00FB802EF80
:1053F0002AF00501306702EF2AF00FB802EF2AF019
:1054000071EF33F081B817EF2AF0FFEC2DF00501B2
:105410002F51020A02E017EF2AF0602F17EF2AF04F
:105420005FC560F50501010E306F3C0E316FB4EFC2
:105430000DF018C100F119C101F11AC102F11BC12F
:1054400003F1000E046F000E056F010E066F000ED3
:10545000076F05EC2CF029A144EF2AF02051D8B4B5
:1054600044EF2AF018C100F119C101F11AC102F18B
:105470001BC103F1000E046F000E056F0A0E066FCC
:10548000000E076F05EC2CF012000101045100130F
:1054900005510113065102130751031312000101B4
:1054A000186B196B1A6B1B6B12002AC182F4040172
:1054B000300E82276DEC0EF02BC182F40401300E09
:1054C00082276DEC0EF02CC182F40401300E82278D
:1054D0006DEC0EF02DC182F40401300E82276DECCC
:1054E0000EF02EC182F40401300E82276DEC0EF016
:1054F0002FC182F40401300E82276DEC0EF030C112
:1055000082F40401300E82276DEC0EF031C182F47A
:105510000401300E82276DEC0EF032C182F40401DA
:10552000300E82276DEC0EF033C182F40401300E90
:1055300082276DEC0EF012002FC182F40401300EB0
:1055400082276DEC0EF030C182F40401300E822708
:105550006DEC0EF031C182F40401300E82276DEC47
:105560000EF032C182F40401300E82276DEC0EF091
:1055700033C182F40401300E82276DEC0EF012006C
:10558000060E1D6E060E1E6E060E1F6E1D2EC6EF3B
:105590002AF01E2EC6EF2AF01F2EC6EF2AF08B84AB
:1055A000020E1D6E020E1E6E020E1F6E1D2ED6EF17
:1055B0002AF01E2ED6EF2AF01F2ED6EF2AF08B945B
:1055C00012000101005305E1015303E1025301E11F
:1055D000002BA4EC2BF0CFEC2CF03951006F3A519A
:1055E000016F420E046F4B0E056F000E066F000E2A
:1055F000076FE5EC2BF000C104F101C105F102C118
:1056000006F103C107F118C100F119C101F11AC176
:1056100002F11BC103F107B212EF2BF0D9EC2BF012
:1056200014EF2BF0D4EC2BF000C118F101C119F1EB
:1056300002C11AF103C11BF11200CFEC2CF059C1C9
:1056400000F15AC101F1060E19EC0BF0E8CF04F19C
:10565000070E19EC0BF0E8CF05F1080E19EC0BF072
:10566000E8CF06F1090E19EC0BF0E8CF07F1D4EC06
:105670002BF000C124F101C125F102C126F103C1C3
:1056800027F1290E046F000E056F000E066F000E45
:10569000076FE5EC2BF0EE0E046F430E056F000E66
:1056A000066F000E076FD9EC2BF024C104F125C161
:1056B00005F126C106F127C107F1E5EC2BF000C189
:1056C0001CF101C11DF102C11EF103C11FF1120E37
:1056D00019EC0BF0E8CF04F1130E19EC0BF0E8CF46
:1056E00005F1140E19EC0BF0E8CF06F1150E19ECCC
:1056F0000BF0E8CF07F10D0E006F000E016F000EEA
:10570000026F000E036FE5EC2BF0180E046F000E15
:10571000056F000E066F000E076F05EC2CF01CC124
:1057200004F11DC105F11EC106F11FC107F1D9EC3D
:105730002BF06A0E046F2A0E056F000E066F000E26
:10574000076FD4EC2BF01200BF0EFA6E200E3A6FEA
:10575000396BD8900037013702370337D8B0B5EF2F
:105760002BF03A2FAAEF2BF039073A070353D8B49E
:1057700012000331070B80093F6F03390F0B010F34
:10578000396F80EC5FF0406F390580EC5FF0405D71
:10579000405F396B3F33D8B0392739333FA9CAEF5F
:1057A0002BF04051392712000101F4EC2CF0D8B055
:1057B0001200010103510719346FB7EC2CF0D89097
:1057C0000751031934AF800F12000101346BDBEC79
:1057D0002CF0D8A0F1EC2CF0D8B01200C6EC2CF0D4
:1057E000CFEC2CF01F0E366F07EC2DF00B35D8B038
:1057F000B7EC2CF0D8A00335D8B01200362FF4EF58
:105800002BF034B1DEEC2CF012000101346B0451AA
:105810000511061107110008D8A0DBEC2CF0D8A068
:10582000F1EC2CF0D8B01200086B096B0A6B0B6B13
:1058300007EC2DF01F0E366F07EC2DF007510B5DB6
:10584000D8A42FEF2CF006510A5DD8A42FEF2CF02E
:105850000551095DD8A42FEF2CF00451085DD8A0A4
:1058600042EF2CF00451085F0551D8A0053D095FB7
:105870000651D8A0063D0A5F0751D8A0073D0B5F2F
:10588000D8900081362F1CEF2CF034B1DEEC2CF0D8
:10589000346BDBEC2CF0D8900BEC2DF007510B5D4A
:1058A000D8A45FEF2CF006510A5DD8A45FEF2CF06E
:1058B0000551095DD8A45FEF2CF00451085DD8A014
:1058C0006EEF2CF0003F6EEF2CF0013F6EEF2CF0EE
:1058D000023F6EEF2CF0032BD8B4120034B1DEEC93
:1058E0002CF012000101346BDBEC2CF0D8B012006C
:1058F00010EC2DF0200E366F0037013702370337DA
:1059000011EE33F00A0E376FE7360A0EE75CD8B0B7
:10591000E76EE552372F84EF2CF0362F7CEF2CF01A
:1059200034B12981D890120001010A0E346F200E83
:10593000366F11EE29F03451376F0A0ED890E652C7
:10594000D8B0E726E732372F9FEF2CF0033302332E
:1059500001330033362F99EF2CF0E750FF0FD8A01A
:105960000335D8B0120029B1DEEC2CF0120004513E
:1059700000270551D8B0053D01270651D8B0063D96
:1059800002270751D8B0073D032712000051086FC6
:105990000151096F02510A6F03510B6F120001018F
:1059A000006B016B026B036B12000101046B056B52
:1059B000066B076B12000335D8A012000351800B51
:1059C000001F011F021F031F003FEEEF2CF0013FDD
:1059D000EEEF2CF0023FEEEF2CF0032B342B0325DF
:1059E00012000735D8A012000751800B041F051FB5
:1059F000061F071F043F04EF2DF0053F04EF2DF0B5
:105A0000063F04EF2DF0072B342B0725120000373B
:105A1000013702370337083709370A370B371200C7
:105A20000101296B2A6B2B6B2C6B2D6B2E6B2F6B53
:105A3000306B316B326B336B120001012A510F0B4B
:105A40002A6F2B510F0B2B6F2C510F0B2C6F2D51DD
:105A50000F0B2D6F2E510F0B2E6F2F510F0B2F6F22
:105A600030510F0B306F31510F0B316F32510F0B23
:105A7000326F33510F0B336F120010A806D0899488
:105A8000000EC76E220EC66E05D08984000EC76E4A
:105A9000220EC66E050EE82EFED7120010A802D008
:105AA000898401D08994050EE82EFED712003DECC2
:105AB0002DF09E96C69E000EC96EFF0E9EB602D0B9
:105AC000E82EFCD79E96C69E000EC96EFF0E9EB6AF
:105AD00002D0E82EFCD7C9CFAFF59E96C69E000E29
:105AE000C96EFF0E9EB602D0E82EFCD7C9CFB0F526
:105AF0009E96C69E000EC96EFF0E9EB602D0E82E80
:105B0000FCD7C9CFB1F59E96C69E000EC96EFF0E9A
:105B10009EB602D0E82EFCD7C9CFB2F59E96C69E9F
:105B2000000EC96EFF0E9EB602D0E82EFCD7C9CF7C
:105B3000B3F59E96C69E000EC96EFF0E9EB602D0AD
:105B4000E82EFCD7C9CFB4F59E96C69E000EC96E4E
:105B5000FF0E9EB602D0E82EFCD7C9CFB5F54EECAD
:105B60002DF012003DEC2DF09E96C69E800EC96E63
:105B7000FF0E9EB602D0E82EFCD79E96C69EAFC5FD
:105B8000C9FFFF0E9EB602D0E82EFCD79E96C69E99
:105B9000B0C5C9FFFF0E9EB602D0E82EFCD79E9678
:105BA000C69EB1C5C9FFFF0E9EB602D0E82EFCD737
:105BB0009E96C69EB2C5C9FFFF0E9EB602D0E82EC5
:105BC000FCD79E96C69EB3C5C9FFFF0E9EB602D0F7
:105BD000E82EFCD79E96C69EB4C5C9FFFF0E9EB6A2
:105BE00002D0E82EFCD79E96C69EB5C5C9FFFF0E13
:105BF0009EB602D0E82EFCD74EEC2DF012003DEC04
:105C00002DF09E96C69E070EC96EFF0E9EB602D060
:105C1000E82EFCD79E96C69E000EC96EFF0E9EB65D
:105C200002D0E82EFCD7C9CFAFF59E96C69E000ED7
:105C3000C96EFF0E9EB602D0E82EFCD7C9CFB0F5D4
:105C40009E96C69E000EC96EFF0E9EB602D0E82E2E
:105C5000FCD7C9CFB1F59E96C69E000EC96EFF0E49
:105C60009EB602D0E82EFCD7C9CFB2F54EEC2DF08F
:105C70003DEC2DF09E96C69E21C0C9FFFF0E9EB63C
:105C800002D0E82EFCD79E96C69E000EC96EFF0E6F
:105C90009EB602D0E82EFCD7C9CFB6F54EEC2DF05B
:105CA00012003DEC2DF09E96C69E870EC96EFF0E2B
:105CB0009EB602D0E82EFCD79E96C69EAFC5C9FF01
:105CC000FF0E9EB602D0E82EFCD79E96C69EB0C5AB
:105CD000C9FFFF0E9EB602D0E82EFCD79E96C69E48
:105CE000B1C5C9FFFF0E9EB602D0E82EFCD79E9626
:105CF000C69EB2C5C9FFFF0E9EB602D0E82EFCD7E5
:105D00004EEC2DF03DEC2DF09E96C69E22C0C9FFB4
:105D1000FF0E9EB602D0E82EFCD79E96C69EB6C554
:105D2000C9FFFF0E9EB602D0E82EFCD74EEC2DF038
:105D300012003DEC2DF09E96C69E870EC96EFF0E9A
:105D40009EB602D0E82EFCD79E96C69E000EC96E67
:105D5000FF0E9EB602D0E82EFCD79E96C69E800E01
:105D6000C96EFF0E9EB602D0E82EFCD79E96C69E48
:105D7000800EC96EFF0E9EB602D0E82EFCD79E960E
:105D8000C69E800EC96EFF0E9EB602D0E82EFCD7CE
:105D90004EEC2DF012003DEC2DF09E96C69E870E27
:105DA000C96EFF0E9EB602D0E82EFCD79E96C69E08
:105DB000000EC96EFF0E9EB602D0E82EFCD79E964E
:105DC000C69E000EC96EFF0E9EB602D0E82EFCD70E
:105DD0009E96C69E800EC96EFF0E9EB602D0E82E1D
:105DE000FCD79E96C69E800EC96EFF0E9EB602D050
:105DF000E82EFCD74EEC2DF0120010A82DD03DEC73
:105E00002DF09E96C69E22C0C9FFFF0E9EB602D000
:105E1000E82EFCD79E96C69E450EC96EFF0E9EB616
:105E200002D0E82EFCD74EEC2DF03DEC2DF09E96E6
:105E3000C69E8F0EC96EFF0E9EB602D0E82EFCD70E
:105E40009E96C69E000EC96EFF0E9EB602D0E82E2C
:105E5000FCD74EEC2DF012003DEC2DF09E96C69E28
:105E600022C0C9FFFF0E9EB602D0E82EFCD79E9638
:105E7000C69E010EC96EFF0E9EB602D0E82EFCD75C
:105E80004EEC2DF03DEC2DF09E96C69E910EC96E07
:105E9000FF0E9EB602D0E82EFCD79E96C69EA50E9B
:105EA000C96EFF0E9EB602D0E82EFCD74EEC2DF048
:105EB00012003DEC2DF09E96C69E22C0C9FFFF0E3B
:105EC0009EB602D0E82EFCD79E96C69E810EC96E65
:105ED000FF0E9EB602D0E82EFCD74EEC2DF012003D
:105EE0003DEC2DF09E96C69E22C0C9FFFF0E9EB6C9
:105EF00002D0E82EFCD79E96C69E010EC96EFF0EFC
:105F00009EB602D0E82EFCD74EEC2DF012003DECF0
:105F10002DF09E96C69E910EC96EFF0E9EB602D0C3
:105F2000E82EFCD79E96C69EA50EC96EFF0E9EB6A5
:105F300002D0E82EFCD74EEC2DF012003DEC2DF0F7
:105F40009E96C69E910EC96EFF0E9EB602D0E82E9A
:105F5000FCD79E96C69E000EC96EFF0E9EB602D05E
:105F6000E82EFCD74EEC2DF012000501256B266BB8
:105F7000276B286B899A400EC76E200EC66E9E96C0
:105F8000C69E030EC96EFF0E9EB602D0E82EFCD749
:105F90009E96C69E27C5C9FFFF0E9EB602D0E82E6C
:105FA000FCD79E96C69E26C5C9FFFF0E9EB602D0A0
:105FB000E82EFCD79E96C69E25C5C9FFFF0E9EB64D
:105FC00002D0E82EFCD79E96C69EC952FF0E9EB602
:105FD00002D0E82EFCD7898A0F01C950FF0A01E1DF
:105FE000120005012E51130A05E005012E51170A72
:105FF0000CE012000501F00E256FFF0E266F0F0E4C
:10600000276F000E286F0EEF30F00501F00E256FA0
:10601000FF0E266FFF0E276F000E286F899A400E25
:10602000C76E200EC66E9E96C69E030EC96EFF0EEC
:106030009EB602D0E82EFCD79E96C69E27C5C9FF05
:10604000FF0E9EB602D0E82EFCD79E96C69E26C5B1
:10605000C9FFFF0E9EB602D0E82EFCD79E96C69EC4
:1060600025C5C9FFFF0E9EB602D0E82EFCD79E962E
:10607000C69EC952FF0E9EB602D0E82EFCD7898A72
:106080000F01C950FF0A1DE005012E51130A05E05A
:1060900005012E51170A0BE012000501000E256FB5
:1060A000000E266F100E276F000E286F12000501DC
:1060B000000E256F000E266F000E276F010E286F51
:1060C00012000501256B266B276B286B05012E51ED
:1060D000130A05E005012E51170A0CE01200050114
:1060E000000E216F000E226F080E236F000E246F2A
:1060F00083EF30F00501000E216F000E226F800E3D
:10610000236F000E246F21C500F122C501F123C5C4
:1061100002F124C503F125C504F126C505F127C503
:1061200006F128C507F145EC2AF000C125F501C1AB
:1061300026F502C127F503C128F5899A400EC76EDE
:10614000200EC66E9E96C69E030EC96EFF0E9EB6AC
:1061500002D0E82EFCD79E96C69E27C5C9FFFF0E2B
:106160009EB602D0E82EFCD79E96C69E26C5C9FFD5
:10617000FF0E9EB602D0E82EFCD79E96C69E25C581
:10618000C9FFFF0E9EB602D0E82EFCD79E96C69E93
:10619000C952FF0E9EB602D0E82EFCD7898AC9509C
:1061A000FF0A08E104C125F505C126F506C127F55A
:1061B00007C128F5D8900501243323332233213336
:1061C0002151F00B216F2167EDEF30F02267EDEFE9
:1061D00030F02367EDEF30F0246783EF30F00501F6
:1061E000100E2527E86A2623E86A2723E86A282371
:1061F0001200E86A05012E51130A06E005012E512E
:10620000170A0BE0020E120005012851000A03E1F3
:106210002751F00B07E0010E120005012851000A7A
:1062200001E0010E120029C500F12AC501F12BC5BC
:1062300002F12CC503F125C504F126C505F127C5DA
:1062400006F128C507F1D4EC2BF003BF1200F9ECDE
:1062500030F0D8A48BEF31F0899A400EC76E200E33
:10626000C66E9E96C69E060EC96EFF0E9EB602D0E4
:10627000E82EFCD7898A899A9E96C69E020EC96E20
:10628000FF0E9EB602D0E82EFCD79E96C69E27C56E
:10629000C9FFFF0E9EB602D0E82EFCD79E96C69E82
:1062A00026C5C9FFFF0E9EB602D0E82EFCD79E96EB
:1062B000C69E25C5C9FFFF0E9EB602D0E82EFCD7AC
:1062C0009E96C69E000EC96EFF0E9EB602D0E82EA8
:1062D000FCD7898A899A9E96C69E050EC96EFF0EC6
:1062E0009EB602D0E82EFCD79E96C69EC952FF0EDF
:1062F0009EB602D0E82EFCD7C9B074EF31F0898A7F
:106300000501100E2527E86A2623E86A2723E86A94
:10631000282313EF31F01200899A400EC76E200E29
:10632000C66E9E96C69E060EC96EFF0E9EB602D023
:10633000E82EFCD7898A899A9E96C69EC70EC96E9A
:10634000FF0E9EB602D0E82EFCD7898A0501256B88
:10635000266B276B286B1200899A400EC76E200EA1
:10636000C66E9E96C69E050EC96EFF0E9EB602D0E4
:10637000E82EFCD79E96C69EC952FF0E9EB602D04E
:10638000E82EFCD7C9CF37F5898A1200899A400ECA
:10639000C76E200EC66E9E96C69EB90EC96EFF0EC3
:1063A0009EB602D0E82EFCD7898A1200899A400E48
:1063B000C76E200EC66E9E96C69EAB0EC96EFF0EB1
:1063C0009EB602D0E82EFCD7898AFF0EE82EFED7B3
:1063D0001200F9EC30F0D8A41200899A400EC76E72
:1063E000200EC66E9E96C69E030EC96EFF0E9EB60A
:1063F00002D0E82EFCD79E96C69E27C5C9FFFF0E89
:106400009EB602D0E82EFCD79E96C69E26C5C9FF32
:10641000FF0E9EB602D0E82EFCD79E96C69E25C5DE
:10642000C9FFFF0E9EB602D0E82EFCD79E96C69EF0
:10643000C952FF0E9EB602D0E82EFCD7898A0F0102
:10644000C950FF0AD8A4E4EF32F00501FE0E376F01
:1064500057EC2DF0AFC538F5B0C539F5B1C53AF5F3
:10646000B2C53BF5B3C53CF5B4C53DF5B5C53EF584
:106470000784B6C166F1B7C167F1B8C168F1B9C1A7
:1064800069F14BC14FF14CC150F14DC151F14EC1B9
:1064900052F157C159F158C15AF1D8EC20F000C15E
:1064A0003FF501C140F502C141F503C142F50501C7
:1064B000616762EF32F0626762EF32F0636762EF4A
:1064C00032F0646766EF32F073EF32F061C504F1C9
:1064D00062C505F163C506F164C507F1D4EC2BF084
:1064E00003BFE4EF32F059C143F55AC144F5B9C5D1
:1064F00045F5BAC546F507940501110E326F899A24
:10650000400EC76E200EC66E9E96C69E060EC96EC3
:10651000FF0E9EB602D0E82EFCD7898A899A9E96F5
:10652000C69E020EC96EFF0E9EB602D0E82EFCD7A4
:106530009E96C69E27C5C9FFFF0E9EB602D0E82EC6
:10654000FCD79E96C69E26C5C9FFFF0E9EB602D0FA
:10655000E82EFCD79E96C69E25C5C9FFFF0E9EB6A7
:1065600002D0E82EFCD725EE37F0322F02D0C4EF50
:1065700032F09E96C69EDECFC9FFFF0E9EB602D0B9
:10658000E82EFCD7B5EF32F0898A899A9E96C69E8E
:10659000050EC96EFF0E9EB602D0E82EFCD79E9661
:1065A000C69EC952FF0E9EB602D0E82EFCD7C9B0D7
:1065B000CFEF32F0898A0501100E2527E86A2623DD
:1065C000E86A2723E86A2823120021C500F122C5C2
:1065D00001F123C502F124C503F1899A400EC76E6B
:1065E000200EC66E9E96C69E0B0EC96EFF0E9EB600
:1065F00002D0E82EFCD79E96C69E02C1C9FFFF0EB0
:106600009EB602D0E82EFCD79E96C69E01C1C9FF59
:10661000FF0E9EB602D0E82EFCD79E96C69E00C105
:10662000C9FFFF0E9EB602D0E82EFCD79E96C69EEE
:10663000C952FF0E9EB602D0E82EFCD725EE37F0E9
:106640000501100E326F9E96C69EC952FF0E9EB671
:1066500002D0E82EFCD7C9CFDEFF322F23EF33F074
:10666000898A1200899A400EC76E200EC66E9E96C9
:10667000C69E900EC96EFF0E9EB602D0E82EFCD7C5
:106680009E96C69E000EC96EFF0E9EB602D0E82EE4
:10669000FCD79E96C69E000EC96EFF0E9EB602D017
:1066A000E82EFCD79E96C69E000EC96EFF0E9EB6C3
:1066B00002D0E82EFCD79E96C69EC952FF0E9EB60B
:1066C00002D0E82EFCD7C9CF2DF59E96C69EC952A2
:1066D000FF0E9EB602D0E82EFCD7C9CF2EF5898AD0
:1066E0001200C0EC2AF0B9C5E8FFD70802E3C0ECFD
:1066F0002AF0B9C5E8FFC80802E3C0EC2AF0B9C522
:10670000E8FFB90802E3C0EC2AF0B9C5E8FFAA081F
:1067100002E3C0EC2AF0B9C5E8FF9B0802E3C0EC35
:106720002AF0FFEC2DF0C6EC31F0F29CF29E8B9437
:10673000C69AC2909482948C720ED36ED3A4FED764
:1067400089968A909390FF0EE8CF00F0E82EFED74E
:10675000002EFCD78150F294F29A9E909D909E92CA
:106760009D92F298F292F290F286F28E0300FF0070
:10BF0000E844F926000C160C2B0C3F0C520C640C68
:10BF1000760C860C960CA50CB30CC10CCF0CDC0C6B
:06BF2000E80CF40C000C1B
:0200000400F00A
:0100C800FE39
:00000001FF
